:0200000480007A
:10000000B72F0000938F0F8073900F306F00400365
:100010001300000013000000130000001300000094
:100020001300000013000000130000001300000084
:100030001300000013000000130000001300000074
:100040009702000093824211739052309300000097
:10005000130100009301000013020000930200004E
:100060001303000093030000130400009304000036
:10007000130500009305000013060000930600001E
:100080001307000093070000130800009308000006
:100090001309000093090000130A0000930A0000EE
:1000A000130B0000930B0000130C0000930C0000D6
:1000B000130D0000930D0000130E0000930E0000BE
:1000C000130F0000930F000097110200938101D0DD
:1000D0001705020013050553979503009385457A8C
:1000E00013060000EF00001A1705020013058544EF
:1000F000970502009385454D13060000EF00801818
:1001000017A503001305057897B503009385457778
:1001100037B6ABAB1306B6BAEF00C01617B1030083
:1001200013014176EF8050679392120093D2120030
:100130009382D2FF638A02008322010013014100EF
:100140006F0000177300203083220100130141006B
:10015000730020301301C1FF23205100F32220340B
:10016000E3C402FC8322010013014100130141F8A2
:1001700023221100232421002326310023284100BB
:10018000232A5100232C6100232E71002320810299
:10019000232291022324A1022326B1022328C10293
:1001A000232AD102232CE102232EF1022320010570
:1001B0002322110523242105232631052328410567
:1001C000232A5105232C6105232E71052320810745
:1001D000232291072324A1072326B1072328C1073F
:1001E000232AD107232CE107232EF107732520347E
:1001F000F3251034130601006F000000731015344E
:1002000083204100032181008321C10003220101D9
:1002100083224101032381018323C10103240102BD
:1002200083244102032581028325C10203260103A1
:1002300083264103032781038327C1030328010485
:1002400083284104032981048329C104032A010569
:10025000832A4105032B8105832BC105032C01064D
:10026000832C4106032D8106832DC106032E010731
:10027000832E4107032F8107832FC1071301C10775
:10028000730020302320C5006376B50013054500B8
:100290006FF05FFF678000000000000000000000BA
:1002A000000000000000000000000000000000004E
:1002B000130101F8232011002322210023243100FF
:1002C0002326410023285100232A6100232C71009A
:1002D000232E8100232091022322A1022324B10294
:1002E0002326C1022328D102232AE102232CF10272
:1002F000232E010323201105232221052324310568
:100300002326410523285105232A6105232C710545
:10031000232E8105232091072322A1072324B1073F
:100320002326C1072328D107232AE107232CF1071D
:100330009702020083A2422323A02200F32210345A
:10034000232E5106EF00C03B170102000321C121FB
:10035000032101008322C10773901234B7220000E9
:100360009382028873A00230832001000322C1001F
:100370008322010103234101832381010324C1015D
:100380008324010203254102832581020326C10241
:100390008326010303274103832781030328C10325
:1003A000832801040329410483298104032AC10409
:1003B000832A0105032B4105832B8105032CC105ED
:1003C000832C0106032D4106832D8106032EC106D1
:1003D000832E0107032F4107832F81071301010893
:1003E00073002030970202009382C22123A01200E2
:1003F00023A2220023A4320023A6420023A85200F5
:1004000023AA620023AC720023AE820023A09202D2
:1004100023A2A20223A4B20223A6C20223A8D202CC
:1004200023AAE20223ACF20223AE020323A01205A8
:1004300023A2220523A4320523A6420523A85205A0
:1004400023AA620523AC720523AE820523A092077E
:1004500023A2A20723A4B20723A6C20723A8D20778
:1004600023AAE20723ACF207EF605038170102001D
:100470000321810F032101008322C10773901234ED
:10048000B72200009382028873A00230832001000B
:100490000322C1008322010103234101832381013F
:1004A0000324C10183240102032541028325810223
:1004B0000326C10283260103032741038327810307
:1004C0000328C103832801040329410483298104EB
:1004D000032AC104832A0105032B4105832B8105CF
:1004E000032CC105832C0106032D4106832D8106B3
:1004F000032EC106832E0107032F4107832F810797
:100500001301010873002030970202009382820FCA
:1005100083A0020003A1420083A1820003A2C200C3
:1005200083A2020103A3420183A3820103A4C201A7
:1005300083A4020203A5420283A5820203A6C2028B
:1005400083A6020303A7420383A7820303A8C2036F
:1005500083A8020403A9420483A9820403AAC20453
:1005600083AA020503AB420583AB820503ACC20537
:1005700083AC020603AD420683AD820603AEC2061B
:1005800083AE020703AFC20983AF82076780000012
:1005900073700430130101F823201100232221007D
:1005A000232431002326410023285100232A6100FF
:1005B000232C7100232E8100232091022322A102EB
:1005C0002324B1022326C1022328D102232AE102D7
:1005D000232CF102232E01032320110523222105C0
:1005E000232431052326410523285105232A6105AB
:1005F000232C7105232E8105232091072322A10797
:100600002324B1072326C1072328D107232AE10782
:10061000232CF1079702020083A202F523A02200F7
:10062000232E1106EF308029170102000321C1F3A8
:10063000032101008322C10773901234B722000006
:100640009382028873A00230832001000322C1003C
:100650008322010103234101832381010324C1017A
:100660008324010203254102832581020326C1025E
:100670008326010303274103832781030328C10342
:10068000832801040329410483298104032AC10426
:10069000832A0105032B4105832B8105032CC1050A
:1006A000832C0106032D4106832D8106032EC106EE
:1006B000832E0107032F4107832F810713010108B0
:1006C00073002030737004306F00000073104530E9
:1006D000678000007325403073F04330678000006E
:1006E00097070000938747FE232EB5FE2322C5FA05
:1006F000232635F82320F5F8130505F86780000058
:10070000130101FF23261100EF60100BEF20C051F1
:10071000631805008320C1001301010167800000F8
:100720008320C100130101016F3040199307850038
:100730001307F0FF2322F5002324E5002326F5000C
:100740002328F500232005006780000023280500EA
:10075000678000008327450023A2F50003A78700D8
:1007600023A4E50003A787002322B70023A4B70032
:1007700023A8A50083270500938717002320F500F1
:100780006780000003A605009307F0FF13078500AC
:100790006316F6006F008003138707008327470066
:1007A00083A60700E37AD6FE23A2F50023A4B700B0
:1007B00023A4E5002322B70023A8A5008327050072
:1007C000938717002320F5006780000003270501A9
:1007D000832747006FF05FFD0327450083268500D0
:1007E000832705012324D70003278500832645009E
:1007F0002322D70003A747006316A700032785001D
:1008000023A2E7002328050003A507001305F5FF31
:1008100023A0A70067800000032605049387050036
:10082000630406028325C50003274500B385C50080
:100830002326B50063E6E500832505002326B500E1
:10084000138507006F50805367800000130101FF7C
:100850002324810023261100130405002322910084
:10086000EF30103A83278404635AF004832744024C
:1008700063860704930444026F0000028327840404
:100880009387F7FF2324F404832784046358F0023A
:10089000832744026384070213850400EF30406518
:1008A000E30E05FCEF301012832784049387F7FFD3
:1008B0002324F40483278404E34CF0FC9307F0FF23
:1008C0002324F404EF301037EF30903383274404AF
:1008D000635AF00483270401638607049304040128
:1008E0006F000002832744049387F7FF2322F40458
:1008F000832744046358F0028327040163840702BA
:1009000013850400EF30C05EE30E05FCEF30900B62
:10091000832744049387F7FF2322F40483274404A6
:10092000E34CF0FC9307F0FF2322F404032481003E
:100930008320C10083244100130101016F30902FF7
:10094000630A0508130101FE232C8100130405002E
:10095000232E1100232A910023282101232631016F
:1009600013890500EF30D029832404048325C403B0
:100970008329040013850400EF80403C1307F0FF37
:10098000232C0402B3079540B387F9003385A900EF
:100990002322E4042322A400232434012326F40088
:1009A0002324E404631C09028327040163920704DF
:1009B000EF3050288320C1010324810183244101A9
:1009C000032901018329C10013051000130101024D
:1009D00067800000737004306F000000130504018D
:1009E000EFF0DFD413054402EFF05FD46FF05FFC4B
:1009F00013050401EF30C04F93071000E31AF5FA16
:100A0000EFF01FB96FF0DFFA631605007370043062
:100A10006F000000130101FE232A91002328210109
:100A200023263101232E1100232C8100930405007D
:100A300013890500930906006380050AEF800030E2
:100A400013055505EF50001313040500630E050848
:100A5000930745052320F500232E94022320240527
:100A6000EF30101A832404048325C40303290400EF
:100A700013850400EF80802C9306F0FF232C0402E2
:100A8000B30795403307A900B307F9002322D40424
:100A90002322E4002326F4002324D40413050401B4
:100AA00023242401EFF09FC813054402EFF01FC870
:100AB000EF30501823083405130504008320C101CA
:100AC0000324810183244101032901018329C100F9
:100AD000130101026780000013054005EF508009F3
:100AE0001304050063160500737004306F000000E6
:100AF000232084006FF05FF66316050073700430E6
:100B00006F0000006376B500737004306F00000062
:100B1000130101FF23248100130620001384050024
:100B20009305000023261100EFF01FEE630C050073
:100B3000232C85028320C1000324810013010101BD
:100B400067800000737004306F000000130101FB28
:100B50002326110423248104232291042320210528
:100B6000232E3103232C4103232A5103232861031D
:100B7000232671032326C10063060528638C0526FE
:100B800093072000639CF6000327C503930710001A
:100B90006306F700737004306F00000013890600CD
:100BA0009384050013040500EF30C065631A050047
:100BB0008327C10063860700737004306F00000054
:100BC000EF301004032784038327C403130B0000B2
:100BD000930B20009309F0FF130A0401930A4402C7
:100BE0006364F710630479238327C10063820736A7
:100BF00063160B0013058101EF30404AEF3090037C
:100C0000EF109074EF30C07F832744046394370162
:100C100023220404832784046394370123240404D7
:100C2000EF3050019305C10013058101EF30004AF8
:100C300063160530EF30C07C032784038327C40389
:100C40006304F710EF30007FEF30807B832784044C
:100C50006346F0026F00000313850A00EF3040295D
:100C600063040500EF300056832784049387F7FF61
:100C70002324F404832784046356F000832744026A
:100C8000E39C07FC23243405EF30C07AEF30407733
:100C9000832744046346F0026F00000313050A0033
:100CA000EF30002563040500EF30C0518327440472
:100CB0009387F7FF2322F404832744046356F0004C
:100CC00083270401E39C07FC23223405EF30807660
:100CD000EF20001B130B1000EF30807203278403FA
:100CE0008327C403E370F7F00326040463040612A9
:100CF000631A091E0325840093850400EF50000841
:100D0000832784008326040403274400B387D70085
:100D10002324F40063E4E71083278403832604007C
:100D200003274402938717002324D400232CF402C2
:100D30006300071013054402EF30801B9307100077
:100D40006318F50E6F004014EF30C06E8325C100AC
:100D500013050A00EF20D06CEF30806A83278404EB
:100D60006346F0026F00000313850A00EF3040185D
:100D700063040500EF300045832784049387F7FF61
:100D80002324F404832784046356F0008327440259
:100D9000E39C07FC23243405EF30C069EF30406644
:100DA000832744046346F0026F00000313050A0022
:100DB000EF30001463040500EF30C0408327440483
:100DC0009387F7FF2322F404832744046356F0003B
:100DD00083270401E39C07FC23223405EF30806560
:100DE000EF20000AE31805EEEFF08FFA130B100066
:100DF0006FF09FEE83270504E38407D873700430F7
:100E00006F000000737004306F00000003260404BC
:100E1000631006088327040063860704832784037E
:100E20000327440293871700232CF402E31407F0EE
:100E3000EF304060130510008320C10403248104B7
:100E400083244104032901048329C103032A810364
:100E5000832A4103032B0103832BC10213010105E4
:100E60006780000003254400EF30804C8327840313
:100E7000032744022322040093871700232CF40243
:100E8000E31A07EAE30605FAEFF08FF06FF05FFA76
:100E90000325C40093850400EF40506E83270404AB
:100EA0000327C40083260400B307F0403307F7008C
:100EB0002326E400637ED70403274400B307F7002A
:100EC0002326F40013072000832744026304E90467
:100ED0000327840313071700232CE402E38A07F493
:100EE0006FF05FE50325C40093850400EF401069AF
:100EF000832704040327C40083260400B307F040BB
:100F00003307F7002326E400E37ED7FA6FF0DFFA19
:100F10008327440203278403E30C07FA032784038F
:100F20001307F7FF232CE40203278403130717009A
:100F3000232CE402E38E07EE6FF0DFDF13050400DD
:100F4000EFF0DF90EF10D073130500006FF0DFEECD
:100F5000EF30404E130500006FF01FEE130101FF4C
:100F600023229100930405001305400523248100EA
:100F700023261100EF40104013040500630C050404
:100F8000232C05029307F0FF2322F504130710001A
:100F900013050501232EE4022324F4042322040074
:100FA0002320040023240400232604002320040417
:100FB00023089404EFF08FF713054402EFF00FF7C6
:100FC00093060000130600009305000013050400BB
:100FD000EFF0DFB7130504008320C1000324810074
:100FE00083244100130101016780000063040504AC
:100FF000130101FF232481002322910023261100E5
:10100000232021010329450013040500EF30801E31
:10101000930400006304A9028320C100032481001B
:1010200013850400032901008324410013010101F9
:1010300067800000737004306F0000008327C400D5
:10104000930410009387F7FF2326F400E39607FC30
:10105000930600001306000093050000130504002A
:10106000EFF0DFAE6FF05FFB6302050A63880508EF
:10107000130101FE232C8100232A91002328210142
:1010800023244101232E1100232631019307200040
:101090009384060013090600138A05001304050053
:1010A000639CF6000327C503930710006302F70A49
:1010B000737004306F000000EFF0CFE1032784036A
:1010C0008327C403930905006366F70493040000B3
:1010D00013850900EFF08FDF8320C1010324810114
:1010E0001385040003290101832441018329C100E0
:1010F000032A810013010102678000008327050491
:10110000E38807F6737004306F00000073700430DA
:101110006F00000003260404631E060C83270400EE
:1011200063860712832784031307F0FF9387170052
:10113000232CF402832784046388E70E8327840426
:1011400093041000938717002324F4046FF05FF8D2
:10115000EFF04FD8032784038327C40393090500C6
:101160006360F70603260404E30A06FA0325C400B5
:1011700093050A00EF409040832704040327C4002E
:1011800083260400B307F0403307F7002326E4006A
:101190006378D70003274400B307F7002326F40041
:1011A00093072000E390F4F883278403E38C07F689
:1011B000832784039387F7FF232CF4026FF09FF6B5
:1011C00003260404E30C06F40325C40093050A0077
:1011D000EF40D03A832704040327C4008326040089
:1011E000B307F0403307F7002326E400E364D7FA9F
:1011F0006FF09FFBE39C04F60325840093050A002F
:10120000EF40D0378327840083260404032744005B
:10121000B387D7002324F400E3E6E7F08327040034
:101220002324F4006FF01FF083274402930410007E
:10123000E38007EA13054402EF20904BE30A05E838
:10124000E30809E8232099006FF09FE80325440094
:10125000EF30000E232204006FF0DFEC6302050A7A
:101260008327050463860700737004306F00000055
:1012700083270500638A0708130101FE232C8100E0
:10128000232A91001304050023282101232631017C
:10129000232E110013890500EFF0CFC30327840329
:1012A0008327C40393090500930400006376F702C3
:1012B000832784031307F0FF93871700232CF4027E
:1012C00083278404638AE70483278404930410003B
:1012D000938717002324F40413850900EFF00FBF50
:1012E0008320C10103248101138504000329010126
:1012F000832441018329C10013010102678000009A
:10130000737004306F00000083274500E38607F602
:10131000737004306F000000832744026396070057
:10132000930410006FF05FFB13054402EF20503C64
:10133000E30805FEE30609FE930710002320F900E9
:101340006FF01FFE130101FC232E1102232C8102DA
:10135000232A910223282103232631032324410336
:10136000232251032326C10063060528638C05262A
:10137000938A06009389050013040500EF20906806
:10138000631A05008327C100638607007370043069
:101390006F000000EF30C006832784036394071CAE
:1013A0008327C1006380071013058101EF20104FD0
:1013B0009304F0FF13094402130A0401EF3080077D
:1013C000EF108078EF30C0038327440463949700C4
:1013D00023220404832784046394970023240404B1
:1013E000EF3040059305C10013058101EF20104E39
:1013F00063100524EF30C00083278403638A070A43
:10140000EF304003EF20D07F832784046346F0024F
:101410006F00000313050900EF20902D6304050001
:10142000EF20505A832784049387F7FF2324F40482
:10143000832784046356F00083274402E39C07FC5F
:1014400023249404EF20107FEF20907B8327440413
:101450006346F0026F00000313050A00EF205029D5
:1014600063040500EF201056832744049387F7FF99
:101470002322F404832744046356F00083270401E5
:10148000E39C07FC23229404EF20D07AEF10501F36
:10149000EF201077832784036396070C8327C1000E
:1014A000E39E07F0EF201079130500006F00800F16
:1014B000EF20507883270400638807108325C1003C
:1014C00013050900EF20C075EF2090738327840473
:1014D0006346F0026F00000313050900EF2050215E
:1014E00063040500EF20104E832784049387F7FFE1
:1014F0002324F404832784046356F00083274402E2
:10150000E39C07FC23249404EF20D072EF20506F5B
:10151000832744046346F0026F00000313050A00AA
:10152000EF20101D63040500EF20D04983274404F9
:101530009387F7FF2322F404832744046356F000C3
:1015400083270401E39C07FC23229404EF20906E80
:10155000EF10101363040508EF20906A83278403BB
:10156000E38E07F293850900130504008324C40069
:10157000EFF08FAA63940A088327840303270400EB
:101580009387F7FF232CF40263160700EF20D07136
:101590002322A4008327040163920708EF209069A7
:1015A000130510008320C103032481038324410316
:1015B000032901038329C102032A8102832A4102EC
:1015C0001301010467800000EF20906303254400AD
:1015D000EF201046EF2010666FF05FEEEFE05FFB4C
:1015E0006FF09FF783270504E38407D873700430F6
:1015F0006F000000737004306F0000008327440206
:1016000023269400E38C07F813054402EF20500EC4
:10161000E30605F8EFE0DFF76FF05FF8130504016C
:10162000EF20100D93071000E31AF5F66FF09FFE00
:1016300013050400EFF08FA1EF10900413050000D4
:101640006FF05FF663000506130101FF232481009C
:101650002320210123261100232291008324450009
:101660001389050013040500EF20D0386380A4041B
:1016700093060000130609009305000013050400FB
:10168000EFF05FCC93071000630CF5028320C100DC
:101690000324810083244100032901001301010177
:1016A00067800000737004306F0000008327C4005F
:1016B00013051000938717002326F4006FF01FFD19
:1016C0008327C400938717002326F4006FF01FFCC4
:1016D000630805066386050C130101FE232C8100B7
:1016E000232A9100232821012326310123244101AB
:1016F00013040500232E1100130906009389050029
:10170000EFE05FFD83278403130A050093040000C4
:10171000639C070213050A00EFE05FFB8320C10111
:10172000032481011385040003290101832441015D
:101730008329C100032A8100130101026780000090
:10174000737004306F000000032604046304060273
:101750008325C40083274400B385C5002326B40035
:1017600063E6F500832504002326B40013850900F1
:10177000EF40C060832784031307F0FF9387F7FFD0
:10178000232CF402832744046384E7028327440460
:1017900093041000938717002322F4046FF09FF73F
:1017A00083270504E38A07F2737004306F0000009A
:1017B0008327040163960700930410006FF09FF5E0
:1017C00013050401EF20C072E30805FEE30609FEDD
:1017D000930710002320F9006FF01FFE6306050831
:1017E00083270504638A050863840708130101FE43
:1017F000232C8100232A9100232821012324410145
:1018000013040500232E110023263101138A05003D
:10181000EFE05FEC832784031309050093040000C5
:10182000638E07008329C40093050A001305040092
:10183000EFE09FFE930410002326340113050900F6
:10184000EFE0DFE88320C101032481011385040058
:1018500003290101832441018329C100032A810056
:101860001301010267800000737004306F000000F4
:10187000737004306F000000E38C07FE7370043057
:101880006F00000063160500737004306F000000E5
:10189000130101FF232481001304050023261100F6
:1018A000EF20103603248403EF20D0388320C100BA
:1018B0001305040003248100130101016780000067
:1018C00063160500737004306F000000130101FF00
:1018D000232611002324810013040500EF20503239
:1018E000832784030324C4033304F440EF2090349B
:1018F000130504008320C1000324810013010101AA
:1019000067800000630605000325850367800000EB
:10191000737004306F0000006308050497870300AC
:10192000938747F203A747006304E50403A7C700B2
:101930006302E50803A74701630AE50603A7C70199
:101940006302E50603A74702630AE50403A7C7028B
:101950006302E50403A74703630AE50203A7C7037D
:101960006302E5026F400039737004306F000000BD
:101970001307000013173700B387E70023A0070001
:101980006F404037130770006FF0DFFE13076000F1
:101990006FF05FFE130750006FF0DFFD130740008C
:1019A0006FF05FFD130730006FF0DFFC13072000BE
:1019B0006FF05FFC130710006FF0DFFB0325C50419
:1019C000678000002326B5046780000003450505F5
:1019D00067800000630805000325850313351500A3
:1019E00067800000737004306F000000630C050016
:1019F000832785030325C5033305F54013351500FB
:101A000067800000737004306F0000009787030048
:101A1000938747E303A707006300070403A7870032
:101A20006308070403A707016308070403A78701E6
:101A30006308070403A707026308070403A78702D4
:101A40006308070403A70703630C070403A78703BE
:101A500063040704678000001307000013173700B2
:101A6000B387E70023A0B70023A2A7006780000088
:101A7000130710006FF09FFE130720006FF01FFE8A
:101A8000130730006FF09FFD130740006FF01FFD3C
:101A9000130750006FF09FFC130770006FF01FFCDE
:101AA000130760006FF09FFB97870300938787D928
:101AB00003A747006300E50403A7C7006306E50426
:101AC00003A747016306E50403A7C7016306E5040E
:101AD00003A747026306E50403A7C7026306E504FC
:101AE00003A74703630AE50403A7C7036302A70428
:101AF000678000001307000013173700B387E70063
:101B000023A0070067800000130710006FF0DFFEBE
:101B1000130720006FF05FFE130730006FF0DFFD4A
:101B2000130740006FF05FFD130750006FF0DFFCFC
:101B3000130770006FF05FFC130760006FF0DFFBAE
:101B4000130101FF2324810023229100232021017E
:101B500013040500232611009384050013090600D1
:101B6000EF20100A032744049307F0FF6314F700E3
:101B700023220404032784049307F0FF6314F7006F
:101B800023240404EF20100B83278403639A0700A7
:101B9000130609009385040013054402EF208024F6
:101BA000EF20100683278404635AF004832744023D
:101BB00063860704930444026F00000283278404B1
:101BC0009387F7FF2324F404832784046358F002E7
:101BD000832744026384070213850400EF20403109
:101BE000E30E05FCEF20005E832784049387F7FF54
:101BF0002324F40483278404E34CF0FC9307F0FFD0
:101C00002324F404EF201003EF20807F8327440473
:101C1000635AF004832704016386070493040401D4
:101C20006F000002832744049387F7FF2322F40404
:101C3000832744046358F002832704016384070266
:101C400013850400EF20C02AE30E05FCEF20805727
:101C5000832744049387F7FF2322F4048327440453
:101C6000E34CF0FC9307F0FF2322F40403248100EB
:101C70008320C100832441000329010013010101D5
:101C80006F20407B63020504130101FD232E310107
:101C9000232C410123261102138A070023248102E9
:101CA0002322910223202103232A510123286101A9
:101CB00023267101930790009309070063FAE70058
:101CC000737004306F000000737004306F00000008
:101CD000130B05009384050013090600938B06007F
:101CE000930A08006302082C13050006EF30906881
:101CF000130405006302052A13192900232855033C
:101D0000130609009305500A13850A00EF400019D5
:101D100003C70400832704031309C9FF230AE4024D
:101D200003C70400338927011379C9FF6306070E2F
:101D300083C71400A30AF40283C71400638E070C40
:101D400083C72400230BF40283C724006386070C97
:101D500083C73400A30BF40283C73400638E070AE1
:101D600083C74400230CF40283C744006386070A38
:101D700083C75400A30CF40283C75400638E070882
:101D800083C76400230DF40283C7640063860708D9
:101D900083C77400A30DF40283C77400638E070623
:101DA00083C78400230EF40283C78400638607067A
:101DB00083C79400A30EF40283C79400638E0704C4
:101DC00083C7A400230FF40283C7A400638607041B
:101DD00083C7B400A30FF40283C7B400638E070265
:101DE00083C7C4002300F40483C7C40063860702CA
:101DF00083C7D400A300F40483C7D400638E070014
:101E000083C7E4002301F40483C7E400638607006A
:101E100083C7F400A301F404930A440013850A0065
:101E2000A30104042326340323283405232A0404AD
:101E3000EFE0DF9113058401EFE05F919307A000CD
:101E4000B3873741232C040423288400232CF40077
:101E50002322840223220404232E040413860B006D
:101E600093050B0013050900EFE09F872320A400D2
:101E700063040A0023208A007370043017E901000C
:101E80001309C96C8327090097E401009384C46D8A
:101E9000638C070003A7040083A70400832747047B
:101EA000938717002322F70417E701001307C76A77
:101EB000832707009387170097E6010023AEF66893
:101EC00083A70400638E070E8327090017EB010028
:101ED000130B0B7B639C070083A7040083A7C70237
:101EE00063E6F90097E7010023A0876897E7010000
:101EF0009387C76483A7070017E7010013074765A7
:101F00000325C402032707009387170097E6010003
:101F100023A6F6622324F4046376A70097E7010062
:101F200023A8A76293054001EF60506193850A00E2
:101F30003305AB00EFE01F828327090063880700A9
:101F400083A7040083A74704639C0708832709002D
:101F500013041000638A070083A7040083A7C70245
:101F600063F43701EFE0CFE2130504008320C102E0
:101F70000324810283244102032901028329C10130
:101F8000032A8101832A4101032B0101832BC10014
:101F9000130101036780000013850A00EF3090559C
:101FA0001304F0FF6FF05FFC13152600EF30903C38
:101FB000930A0500E31A05D21304F0FF6FF0DFFA6D
:101FC00097E7010023A2875A032707009307100011
:101FD000630AF70217EB0100130B8B6A6FF01FF116
:101FE00003A7040083A60400832747049387F7FF11
:101FF0002322F70483A74604E39A07F473600430AE
:102000006FF0DFF4130A000017EB0100130B4B67AE
:10201000930BA00013050A0093054001EF601052D6
:10202000130A1A003305AB00EFE04FF0E3147AFF18
:1020300097EB0100938B4B7113850B00EFE00FEFD3
:1020400017EA0100130A8A7113050A00EFE00FEE88
:1020500017E501001305C571EFE04FED17E501002D
:1020600013054572EFE08FEC17E501001305C5720B
:10207000EFE0CFEB97E7010023A6774F97E701004A
:1020800023A0474F6FF09FE6130101FF2324810037
:10209000232611002322910023202101130405008F
:1020A0007370043097E401009384444A83A70400CA
:1020B000639E07106318040097E701009387C74ADF
:1020C00003A407001309440013050900EFE0CFF053
:1020D000832784026386070013058401EFE0CFEFB6
:1020E0009305090017E501001305C569EFE08FE6C8
:1020F00097E701009387874603A7070097E701004A
:102100009387C74383A707001307170097E60100CB
:1021100023A6E64403A704009387170097E601006F
:1021200023AEF640630C070097E701009387C7438F
:1021300003A7070003274704631C070E83A70400B7
:10214000638A070697E701009387074203A7070002
:10215000630287107370043003A704006318070834
:1021600017E70100130707408326070083A6060030
:102170006392060A1307F0FF97E6010023AEE63AE2
:1021800003A704006308070203A707000327470407
:102190006302070203A7070083A6070083274704FB
:1021A0009387F7FF2322F70483A74604639407006D
:1021B000736004308320C100032481008324410024
:1021C00003290100130101016780000097E7010066
:1021D0009387873903A7070083A70700832747044E
:1021E000938717002322F7046FF0DFEC83A6070024
:1021F00003A7070003A746041307170023A2E6045A
:1022000017E70100130707368326070083A6060099
:10221000E38206F6032707000327C7000327C7004A
:102220000327470097E6010023A8E6306FF05FF52B
:1022300003A7070083A60700832747049387F7FFB8
:102240002322F70483A74604E39A07EE7360043061
:102250006FF0DFEE97E701009387C72D83A7070094
:1022600063860700737004306F0000000324810050
:102270008320C100832441000329010013010101CF
:102280006FE00FB16304050C17E701001307C72DBA
:1022900083260700930700006386A60A130101FF47
:1022A000232611002324810023229100737004301F
:1022B00097E601009386862983A70600638C0700B2
:1022C0000326070083270700832746049387170008
:1022D0002322F60483A70600930405000324450186
:1022E000638807008327070083A7470463940706D2
:1022F00097E701009387072783A70700638C87066A
:1023000097E701009387C72583A7070063848706A3
:1023100097E70100938747486306F40497E70100B5
:1023200093874746630CF402930710008320C10093
:102330000324810083244100138507001301010158
:102340006780000013850700678000007370043009
:102350006F000000EF6090346FF09FF9930740002A
:102360006FF0DFFC83A7840293B7170093872700E1
:102370006FF0DFFB930720006FF05FFB737004309A
:1023800097E701009387871C03A7070063160702DE
:102390006304050483A707000325C502638C0700B7
:1023A00097E701009387471C03A70700032747040B
:1023B000631C07026780000017E701001307C71AB4
:1023C000832607000327070003A746041307170007
:1023D00023A2E604E31005FC17E701001307C71862
:1023E000032507006FF01FFB03A7070083A6070064
:1023F000832747049387F7FF2322F70483A7460424
:10240000E39A07FA7360043067800000130101FF4C
:10241000232481001304050023261100EFE08FAB75
:102420006318040097E701009387071403A40700CB
:102430000324C402EFE08FA98320C1001305040028
:1024400003248100130101016780000093079000BD
:1024500063F6B700737004306F000000130101FED3
:10246000232C8100232E1100232A910023282101EF
:102470002326310123244101130405007370043025
:1024800017E901001309890C8327090063920710DB
:102490006300041283270405638EF50A17E7010021
:1024A0001307870C63F0B70283260700638E86123A
:1024B000032707008324C702B3B4950093C4140014
:1024C0006F00000183240700B384844093B4140098
:1024D0000327C4026386E70E832784012328B404FC
:1024E00063C807009307A000B385B740232CB4004E
:1024F00093172700B387E7000327440197E90100FA
:102500009389091893972700B387F9006310F7049C
:10251000130A440013050A00EFE00FAC97E701002F
:10252000938707030325C40283A7070063F6A70068
:1025300097E7010023AEA70093054001EF6010006C
:1025400093050A003385A900EFE0CFA0638404005F
:10255000EFE00F8483270900638C070097E70100F1
:102560009387870083A7070083A74704639E070418
:102570008320C10103248101832441010329010136
:102580008329C100032A8100130101026780000032
:1025900097E70100938747FD03A7070083A707007C
:1025A00083274704938717002322F704E31404EEDC
:1025B00097E70100938747FB03A407006FF09FEDA7
:1025C0002326B4026FF05FF1032481018320C1014F
:1025D00083244101032901018329C100032A8100C9
:1025E000130101026F60900B930400006FF05FEE27
:1025F000630A0508130101FE232A910097E40100F4
:10260000938484F683A70400232E1100232C8100D9
:1026100023282101232631016388A7047370043025
:1026200017E90100130989F283270900638C070069
:1026300003A7040083A70400832747049387170098
:102640002322F7040327450197E701009387C71466
:10265000630EF702832709006388070083A704003D
:1026600083A74704639E07088320C10103248101D7
:1026700083244101032901018329C10013010102BF
:1026800067800000737004306F00000083278502AC
:1026900017E701001307C70DE38EE7FAE39C07FA7B
:1026A000930945001304050013850900EFE0CF925C
:1026B00097E701009387C7E90325C40283A70700B2
:1026C00063F6A70097E7010023A4A7E8930540015C
:1026D000EF60C06697E70100938787FA3385A7000C
:1026E00093850900EFE00F8783A704000327C40246
:1026F00083A7C702E360F7F6EFD09FE96FF09FF57D
:10270000032481018320C1018324410103290101A4
:102710008329C100130101026F604078630205063E
:10272000130101FE232C8100232A9100232631016D
:1027300013040500232E110023282101EFD09FF957
:102740000327440197E701009387070593090500D4
:1027500093040000630AF70213850900EFD01FF706
:102760008320C10103248101138504000329010191
:10277000832441018329C100130101026780000005
:10278000737004306F0000008327840217E5010096
:10279000130505FEE382A7FCE39007FC97E7010021
:1027A000938747D983A707006394070697E701003B
:1027B000938787DB83A707008324C402130944009F
:1027C00083A7C70213050900B3B4F400EFE0CF807C
:1027D00097E701009387C7D70325C40283A70700A3
:1027E00093C4140063F6A70097E7010023A2A7D6BD
:1027F00093054001EF60805497E70100938747E815
:10280000930509003385A700EFD0DFF46FF0DFF404
:1028100093058401EFD01FF46FF01FF4130101FE44
:1028200037150000232E1100232C8100232A91004C
:102830002328210123263101232441012322510190
:1028400023206101EF300033630805229304050063
:1028500013050006EF30003213040500630405265B
:10286000371600009305500A2328950213850400AB
:10287000EF30C06283240403B71700009387C7FFBB
:10288000B384F400B7474C4593879744130A440038
:10289000232AF40213050A00230C0402A3010404F2
:1028A0002326040223280404232A0404EFD01FEA69
:1028B00013058401EFD09FE99307A000232C0404A3
:1028C00093F4C4FF23288400232CF40023228402E1
:1028D00023220404232E040413060000971500008D
:1028E0009385C5EA13850400EFD09FDF2320A40061
:1028F0007370043017E90100130949C583270900E3
:1029000097E40100938444C6638C070003A7040086
:1029100083A7040083274704938717002322F70423
:1029200017E70100130747C38327070093871700A2
:1029300097E6010023A2F6C283A704006388070A72
:102940008327090097E90100938989D3639C0700D5
:1029500083A7040083A7C7026396070097E70100D7
:1029600023A487C097E70100938747BD03A707000B
:1029700097E601009386C6BD8327C40283A606009E
:102980001307170017E60100232AE6BA2324E404FC
:1029900063F6F60017E70100232CF7BA139527001A
:1029A0003305F5001315250093050A003385A900AA
:1029B000EFD05FDA832709006388070083A704004C
:1029C00083A74704639E070C8327090063840700DD
:1029D00083A70400EF20100993071000630AF51085
:1029E000631C0508737004306F00000097E7010056
:1029F00023AC87B6032707009307100097E901006F
:102A0000938909C8E310F7F6938A090017EB0100D0
:102A1000130B8BD313850A00938A4A01EFD01FD181
:102A2000E31A5BFF17E50100130505D2EFD01FD0B5
:102A300097EA0100938A8AD213850A00EFD01FCF4C
:102A400017E501001305C5D2EFD05FCE17E50100F1
:102A5000130545D3EFD09FCD17E501001305C5D36E
:102A6000EFD0DFCC97E7010023AE67AF97E7010017
:102A700023A857AF6FF01FEF8320C101032481010A
:102A800083244101032901018329C100032A810014
:102A9000832A4100032B010013010102678000001B
:102AA00003A7040083A60400832747049387F7FF46
:102AB0002322F70483A74604E39807F073600430E9
:102AC0006FF09FF0032481018320C10103290101DC
:102AD0008329C100032A8100832A4100032B0100BE
:102AE0001385040083244101130101026F3080200B
:102AF000737004309307F0FF17E70100232EF7A24D
:102B00000324810197E7010023A2A7A48320C10128
:102B100083244101032901018329C100032A810083
:102B2000832A4100032B010097E7010023A407A299
:102B3000130101026FD01F8B7370043097E70100FF
:102B400023A607A06FD05F9C17E701001307879E9D
:102B500083270700938717002320F7006780000072
:102B60007370043097E701009387479E03A707001F
:102B70006318070217E701001307C79D0325070025
:102B800083A70700638C070097E701009387C79D21
:102B900003A70700032747046314070267800000A8
:102BA00017E701001307479C832607000327070048
:102BB00003A746041307170023A2E6046FF09FFB48
:102BC00003A7070083A60700832747049387F7FF1F
:102BD0002322F70483A74604E39207FC73600430C2
:102BE00067800000130101FF2326110023248100C8
:102BF000EFD05FAE97E701009387C79503A4070066
:102C0000EFD0DFAC8320C100130504000324810052
:102C1000130101016780000097E701009387C793C4
:102C200003A5070067800000130101FD23261102A0
:102C3000232481022322910223202103232E310108
:102C4000232C4101232A51012328610123267101EC
:102C500097E701009387078E83A70700639A07060B
:102C600017E701001307078F8327070093871700D3
:102C700097E6010023A0F68E832A0700638A0A0ADA
:102C800097E701009387478B83A707009304000011
:102C900063FEFA0A97E901009389899E17EA010009
:102CA000130A8A8C83270A009306100003A7C70221
:102CB00093172700B387E70093972700B389F9009C
:102CC00083A7090063F4F602930410006F0000026A
:102CD00097E701009387478783A7070093040000C5
:102CE0009387170017E701002320F78697E7010075
:102CF0009387478583A70700638407009304100028
:102D00008320C102032481021385040003290102E8
:102D1000832441028329C101032A8101832A4101BD
:102D2000032B0101832BC100130101036780000005
:102D300017E40100130404838327040083A707001A
:102D40006388070C737004306F00000017E4010003
:102D50001304448197E901009389899217EA0100DD
:102D6000130A8A8017DB0100130B8B7E8327040074
:102D700083A70700638007088327040083A7C70091
:102D800003A9C70083274900930B490013850B0053
:102D900063EAFA06EFD05FA483278902130589014D
:102DA00063840700EFD05FA38327C90203270B00CA
:102DB00093850B00139527003305F50013152500A7
:102DC0003385A9006376F70017D701002322F7782F
:102DD000EFD05F9883270A000327C90283A7C702A1
:102DE000E366F7F8832704009304100083A7070025
:102DF000E39407F89307F0FF17D70100232EF7722B
:102E00006FF05FEA17D701002328F7726FF09FE990
:102E100017D701001307C77483270400032707008F
:102E200097D6010023A0E67417D70100232AF77272
:102E300097D701009387C77083A707009387170070
:102E400017D70100232EF76E8327040083A70700FE
:102E5000639A07009307F0FF17D70100232EF76C42
:102E60006FF01FE28327040083A7C70083A7C70072
:102E700083A7470017D701002320F76C6FF05FE0AE
:102E800097D701009387076B03A707006316070016
:102E9000737004306F000000130101FE232E110037
:102EA000232C8100232A910023282101232631018C
:102EB0002324410123225101232061017370043036
:102EC00097D401009384846803A704006310071259
:102ED00003A707001307F7FF97D6010023ACE664AA
:102EE00083A70700639E070A97D701009387C766E9
:102EF00083A707006386070A97DA0100938A4A7856
:102F000017DA0100130ACA6417D901001309C96549
:102F1000930910006F00C0013385EA00EFD09F8352
:102F2000832709000327C40283A7C7026374F70637
:102F300083A70A0F6380070E83A7CA0F03A4C700E5
:102F400013058401EFD05F89130B440013050B00B8
:102F5000EFD09F888327C40283260A0093050B00C5
:102F6000139527003305F5001315250013070500F9
:102F70003385AA00E3F2F6FA17D70100232AF75C9B
:102F8000EFD04FFD832709000327C40283A7C702A0
:102F9000E360F7FA97D7010023A6375B6FF05FF97C
:102FA0001304000083A70400638C070097D7010077
:102FB0009387875B83A7070083A747046398070469
:102FC000130504008320C1010324810183244101EE
:102FD000032901018329C100032A8100832A4100BA
:102FE000032B0100130101026780000017D70100C5
:102FF00013078757832607000327070003A7460404
:103000001307170023A2E6046FF09FECEF5010693E
:103010006FF01FFB17D4010013040453832704002F
:10302000638C0702832704001309100063860702DC
:10303000EFF09FBF6306050097D7010023A4275137
:10304000832704009387F7FF17D70100232EF74E3D
:1030500083270400E39E07FC97D701009387874EE0
:1030600003A7070093071000E31CF7F2EFD04FD23D
:10307000130410006FF01FF363040502639605004C
:10308000737004306F00000017D701001307874AE0
:1030900083270700638A0700737004306F00000005
:1030A000737004306F000000130101FF23248100BE
:1030B00023261100832607000327050093861600A8
:1030C00017D601002328D64697D601009386864856
:1030D00083A606003304B7002320850063F0E604CE
:1030E0006372E40263F0860297D701009387C747B3
:1030F00003A5070013054500EFD00FEE13050400EC
:10310000EF505051EFF0DFD7630E05008320C10070
:10311000032481001301010167800000E366E4FCE1
:103120006FF05FFC032481008320C10013010101C3
:103130006FD00FC6630E050017D701001307873F36
:103140008327070063880700737004306F00000056
:103150006FD00FC4130101FF232611002324810027
:1031600003270700930705001307170097D60100F0
:1031700023A2E63C97D601009386063F17D70100AD
:103180001307473D0327070003A506003304F70094
:1031900013054500EFD04FE413050400EF509047AE
:1031A000EFF01FCE631A0500032481008320C100C5
:1031B000130101016FD0CFBD8320C1000324810022
:1031C0001301010167800000130101FF2324810026
:1031D0002326110097D701009387C73583A70700DF
:1031E000130400009387170017D701002324F73436
:1031F00097D701009387473683A7070063EEF5143E
:1032000017DE0100130E8E5397D20100938282467F
:103210001304000013070000930F10001303500A5B
:103220006F00C000130ECEFE6384C20F83278EFF93
:1032300093060700E38807FE8327CEFF83A7470096
:10324000232EFEFE6386C71303AFC70083A7470084
:103250003307E500930E0000232EFEFE6380C709AE
:1032600083A8C70093874803232017012322F70070
:1032700083A788042326F7012324F70083A7C80225
:103280002328F70083A70805232C0700232AF7002B
:1032900003A808038347080063986704930708009E
:1032A0009387170083C60700B3850741E38A66FE4C
:1032B00093D525009395050193D50501231EB700ED
:1032C000938E1E0013070702630A1F038327CEFF96
:1032D00083A74700232EFEFEE394C7F983274E0001
:1032E000232EFEFE6FF0DFF793050000231EB700CC
:1032F000938E1E0013070702E31A1FFD3304D40147
:1033000013175400130ECEFE93060700E390C2F38A
:1033100097D701009387072503AE070083270E0088
:103320006396071297D701009387872303AE0700A0
:1033300083270E00639A071C17DE0100130E4E341C
:1033400083274E10639C070283278E11639C0726F8
:103350006304060023200600EFF09FB2130504006B
:103360008320C10003248100130101016780000054
:1033700083274E00232EFEFE6FF01FED83278E1055
:1033800017DF0100130F8F4083A7470017D70100F5
:10339000232CF73E6386E73D83A2C70083A747003F
:1033A000B306D500930E000017D70100232EF73C7B
:1033B000930F40001303500A6382E70983A8C700F4
:1033C0009387480323A0160123A2F60083A788044D
:1033D00023A6F60123A4F60083A7C80223A8F600BB
:1033E00083A7080523AC060023AAF60003A8080358
:1033F00083470800639A6732930708009387170092
:1034000003C70700B3850741E30A67FE93D725008A
:103410009397070193D70701239EF600938E1E0012
:1034200093860602638C123183278E1083A7470090
:1034300017D70100232AF734E392E7F983270E1107
:1034400017D701002322F7346FF05FF783274E0070
:10345000130F8E0083A647002322DE006380E6332D
:10346000B307E50003A7460083A2C600930E000041
:103470002322EE00930F20001303500A6300EF088D
:103480008328C7001387480323A0170123A2E7005E
:1034900003A7880423A6F70123A4E70003A7C80213
:1034A00023A8E70003A7080523AC070023AAE70029
:1034B00003A8080303470800631E672213070800D8
:1034C0001307170083460700B3050741E38A66FE2A
:1034D00013D725001317070113570701239EE70091
:1034E000938E1E00938707026380122383264E006B
:1034F00003A746002322EE00E314EFF80327CE00D3
:103500002322EE006FF0DFF783274E00130F8E00AB
:1035100083A747002322FE00638CE72583A2C70010
:1035200083A74700B306D500930E00002322FE00B8
:10353000930F20001303500A6300FF0883A8C700FD
:103540009387480323A0160123A2F60083A78804CB
:1035500023A6F60123A4F60083A7C80223A8F60039
:1035600083A7080523AC060023AAF60003A80803D6
:103570008347080063986714930708009387170030
:1035800003C70700B3850741E30A67FE93D7250009
:103590009397070193D70701239EF600938E1E0091
:1035A00093860602638A121383274E0083A747007F
:1035B0002322FE00E314FFF88327CE002322FE001F
:1035C0006FF0DFF78327CE1197DE0100938E4E1D3B
:1035D00083A7470017D701002322F71C638AD71758
:1035E00083AFC70083A747003307D500130300004C
:1035F00097D6010023A4F61A130F3000930220007F
:103600009308500A6388D70903A5C70093074503A9
:103610002320A7002322F700832785042326E70120
:103620002324F7008327C5022328F7008327850278
:10363000638407002326570083270505232C0700F2
:10364000232AF7000328050383470800639C170516
:10365000930708009387170083C60700B3850741C7
:10366000E38A16FF93D725009397070193D70701A5
:10367000231EF7001303130013070702638EAF0224
:103680008327CE1183A7470097D6010023A8F61001
:10369000E39CD7F783274E1297D6010023A0F6109C
:1036A0006FF09FF693070000231EF700130313002B
:1036B00013070702E396AFFC33046400E31C06C85B
:1036C0006FF09FC993070000239EF600938E1E00A3
:1036D00093860602E39A12ED17DE0100130E4EFAEE
:1036E00083274E103304D40193165400E38E07C48D
:1036F0006FF0DFC813070000239EE700938E1E00C3
:1037000093870702E39412DF97D70100938747E579
:1037100003AE07003304D4019316540083270E0030
:10372000E38C07C06FF05FDE93070000239EF60076
:10373000938E1E0093860602E39812CF83278E1184
:103740003304D40193165400E38407C06FF09FE75D
:1037500083274E1217D701002322F7046FF05FE88A
:1037600083270E1117D701002320F7026FF0DFC265
:103770008327CE002322FE006FF05FDA8326CE007F
:103780002322DE006FF0DFCD130101FD2322910221
:1037900023202103232E3101232C4101232A51010F
:1037A000232861012326710123261102232481028B
:1037B00097D90100938909D817D90100130949EC59
:1037C00017DA0100130A8AD897DA0100938ACAD956
:1037D00097DB0100938B4BD897D40100938404D8D6
:1037E000130B10006F00000283A709000324491087
:1037F0009387170017D70100232EF7D2EFF04FE879
:10380000631E040083A70400E39007FE83270900DA
:10381000E37AFBFEEFC0DFD76FF0DFFE737004309A
:1038200083270A00639E07048327091103A4C700A6
:1038300013054400EFC05FFA83A70B009387F7FFDF
:1038400017D70100232AF7D083A704009387F7FF37
:1038500017D701002324F7D083270A0063880700C5
:1038600083A70A0083A7470463980702032504037C
:10387000EF20404813050400EF20C0476FF09FF889
:1038800003A70A0083A70A0083274704938717002A
:103890002322F7046FF05FF903A70A0083A60A004A
:1038A000832747049387F7FF2322F70483A746045F
:1038B000E39E07FA736004306FF05FFB97D7010057
:1038C000938747C783A70700639E070E130101FF75
:1038D00023261100232481002322910097D7010081
:1038E00023A207C617D70100130707C883270700BD
:1038F000B7A6A5A59386565A83A7070383A50700F5
:10390000639ED50003A64700631AB60083A687000E
:103910006396C60083A7C700638AD7000325070004
:103920008325070093854503EF30500E17D701001C
:10393000130707C28326070017D40100130444D4D9
:103940006F000002832707006386070883270700AC
:103950009387F7FF97D6010023ACF6BE83260700B6
:1039600093972600B387D70093972700B307F400F7
:1039700083A70700E38807FC0325070093172500AA
:10398000B387A700939727003307F40083264700E7
:1039900093878700B307F40083A44600232297008F
:1039A000638EF40283A7C4008320C1000324810036
:1039B00017D70100232AF7BA83244100130101011C
:1039C000678000009307100017D70100232CF7B67B
:1039D00067800000737004306F00000083A444000F
:1039E00093054001EF5080353305A4002322950054
:1039F0006FF05FFB130101FE23282101232E11002C
:103A0000232C8100232A910023263101130905006C
:103A10007370043097D40100938444B383A70400E7
:103A200017D40100130444B4639C070C6314090009
:103A3000032904009309490013850900EFC0DFD969
:103A4000832789026386070013058901EFC0DFD849
:103A50009385090017D50100130505D4EFC09FCF4A
:103A600083A70400638807008327040083A7470413
:103A70006394070A832704006384270D83A7040047
:103A8000638207067370043083A704006398070EEF
:103A900097D70100938707AD03A707000327070007
:103AA0006310070C9307F0FF17D701002326F7A830
:103AB00083A70400638807028327040083A74704C1
:103AC0006382070203270400832604008327470438
:103AD0009387F7FF2322F70483A746046394070024
:103AE000736004308320C1010324810183244101D8
:103AF000032901018329C10013010102678000002D
:103B000003270400832704008327470493871700B3
:103B10002322F7046FF09FF103270400832604009B
:103B2000832747049387F7FF2322F70483A74604DC
:103B3000E39207F47360043083270400E39027F5D1
:103B400083A704006382070697D701009387879EA7
:103B500083A707006388070A737004306F000000B2
:103B600083A7070083A7C70083A7C70083A74700D1
:103B700017D701002322F79C6FF09FF3032704005F
:103B80008327040083274704938717002322F70421
:103B900097D701009387079D03A707000327070016
:103BA000E30207F06FF0DFFB97D701009387C79A16
:103BB00017D701001307C7AC83A707000327871196
:103BC0006314F7028320C1010324810197D7010008
:103BD00023AC079883244101032901018329C100F3
:103BE0001301010267800000032481018320C101C9
:103BF00083244101032901018329C100130101022A
:103C00006FF0DFCB032481018320C10183244101B4
:103C1000032901018329C100130101026FC05F97CD
:103C20006306050A130101FF2322910097D40100C6
:103C300093848493232021011389050083A5040024
:103C4000232611002324810093858501EFC09FB3B3
:103C500003A5040013054500EFC01FB89307F0FF4C
:103C6000630AF90697D701009387C78E03A407005C
:103C700003A7040083A7070033042401232287003D
:103C8000636EF40697D701009387C78D03A50700DD
:103C900083A5040093854500EFC0DFAE97D70100F0
:103CA0009387878983A707006376F40097D701007D
:103CB00023A487888320C10003248100832441003A
:103CC00003290100130101016780000073700430B3
:103CD0006F00000083A50400032481008320C1003D
:103CE000832441000329010017D501001305C5AA4B
:103CF00093854500130101016FC0DFA597D701002F
:103D00009387078603A507000324810083A5040089
:103D10008320C100832441000329010093854500CD
:103D2000130101016FC01FA6630E050097D70100A4
:103D30009387478083A70700639A07007370043056
:103D40006F000000737004306F000000130101FF6A
:103D50002322910097D401009384048103A70400D7
:103D60009387050083A50400B7060080B3E7D7005A
:103D70002326110023248100232CF700938585013D
:103D800013040600EFC01F9D03A5040013054500A2
:103D9000EFC09FA49307F0FF6304F40297C70100EC
:103DA0009387477B03A507008320C100832441003C
:103DB0003305850003248100130101016F50800544
:103DC00083A50400032481008320C10083244100D3
:103DD00017D501001305459C93854500130101018A
:103DE0006FC05F976308050A130101FF232291004A
:103DF00097C401009384447723202101138905008F
:103E000083A50400232611002324810093858501C6
:103E100013040600EFC01F9403A50400130545001A
:103E2000EFC09F9B93071000630AF40697C7010039
:103E30009387477203A4070003A7040083A7070022
:103E40003304240123228700636EF40697C7010020
:103E50009387477103A5070083A504009385450058
:103E6000EFC05F9297C701009387076D83A7070094
:103E70006376F40097C7010023A0876C8320C100FC
:103E8000032481008324410003290100130101015F
:103E900067800000737004306F00000083A5040089
:103EA000032481008320C1008324410003290100F1
:103EB00017D501001305458E9385450013010101B7
:103EC0006FC05F8997C701009387876903A50700C3
:103ED0000324810083A504008320C10083244100C2
:103EE0000329010093854500130101016FC09F89DB
:103EF000130101FF232611002324810023229100B6
:103F00008327C50003A4C7006304040A9304840143
:103F100013850400EFC05F8C97C70100938787610A
:103F200083A70700639A07089304440013850400DD
:103F3000EFC09F8A97C70100938787610327C40258
:103F400083A7070063F6E70097C7010023A2E76095
:103F500093172700B387E7009397270017C5010041
:103F600013050572938504003305F500EFC08FFE3D
:103F700097C701009387475F83A707000327C40201
:103F80001305000083A7C70263FAE7009307100038
:103F900017C701002328F75A130510008320C1001A
:103FA0000324810083244100130101016780000084
:103FB000737004306F0000009385040017C5010082
:103FC0001305057BEFC00FF96FF09FFA97C701004B
:103FD0009387475683A707006396070073700430E2
:103FE0006F000000130101FF23261100232481002C
:103FF00023229100B70700800324C500B3E7F50032
:104000002320F50063080408EFC00FFD930444006B
:1040100013850400EFC04FFC97C7010093874753F7
:104020000327C40283A7070063F6E70097C70100D0
:1040300023A0E75293172700B387E7009397270041
:1040400017C501001305C5633305F500938504000A
:10405000EFC04FF097C701009387075183A7070070
:104060000327C4021305000083A7C70263FAE70011
:104070009307100017C701002326F74C1305100003
:104080008320C10003248100832441001301010126
:1040900067800000737004306F0000006304050245
:1040A00097C701009387C74903A7070097C7010077
:1040B0009387474A83A707002320E5002322F500C2
:1040C00067800000737004306F0000006304050E09
:1040D000638E050C130101FF2326110023248100A8
:1040E000130705007370043097C8010093880846D1
:1040F00083A708006380070297C701009387C7461C
:1041000083A6070083A7070083A7460493871700A9
:1041100023A2F60417C301001303C34383A70500BA
:10412000032603009306F0FF130400006388D704FE
:1041300017CE0100130ECE4003250E000328070002
:10414000832647006306A800130410006378D60294
:104150003308D640130410006372F80203250E00E2
:10416000B387C74003260300B387D70023A0F50019
:104170002320A7002322C7001304000083A7080000
:10418000638C070097C701009387073E83A707004A
:1041900083A7470463940702130504008320C1002A
:1041A0000324810013010101678000007370043053
:1041B0006F000000737004306F000000EF40104E7D
:1041C0006FF09FFD9307100017C70100232CF736EF
:1041D00067800000630605000325C50467800000B2
:1041E0001305000067800000630405002326B50462
:1041F0006780000097C701009387073703A5070072
:104200006780000097C701009387473483A70700A2
:1042100013051000638C070097C70100938787314F
:1042200003A507001335150013151500678000005E
:10423000630C0508130101FE232A910097C40100B5
:104240009384843283A70400232E1100232C810041
:1042500023282101232631010327C50283A7C70292
:104260006376F7048327850163CC070083A70400E6
:1042700083A6C7029307A000B387D740232CF5007D
:1042800093172700B387E7000327450117C90100EB
:104290001309093F93972700B307F9006308F70252
:1042A00083A7040083A7C7022326F5028320C10148
:1042B0000324810183244101032901018329C100D1
:1042C0001301010267800000678000009309450028
:1042D0001304050013850900EFC00FD083A7040065
:1042E00017C701001307C7260327070083A7C702C4
:1042F0002326F4026376F70017C70100232AF72468
:10430000139527003305F5000324810113152500BB
:104310008320C10183244101938509003305A9004D
:104320008329C10003290101130101026FC08FC25B
:1043300063060502130101FF2326110023248100D7
:104340002322910097C701009387072203A4070047
:10435000630AA400737004306F00000013050000AE
:10436000678000008327440563960700737004305C
:104370006F0000008326C402032704059387F7FF1C
:10438000232AF4046384E600638E0700130500000B
:104390008320C10003248100832441001301010113
:1043A000678000009304440013850400EFC0CFC26F
:1043B0000325040597C701009387871903A7070002
:1043C0009307A000B387A7402326A402232CF40060
:1043D0006376A70097C7010023ACA7169305400199
:1043E000EF40D01597C70100938787293385A70031
:1043F00093850400EFC00FB6130510006FF05FF94E
:104400007370043097C701009387471483A7070090
:104410006380070297C701009387071503A707006A
:1044200083A7070083274704938717002322F704F5
:104430006780000097C701009387471183A7070093
:10444000638C070297C701009387071203A7070031
:10445000032747046302070203A7070083A6070098
:10446000832747049387F7FF2322F70483A7460493
:1044700063940700736004306780000097C70100F1
:104480009387870E03A6070083A6070003A70700EC
:104490009307A00083A6C60203258601B387D740F1
:1044A000232CF7006780000097C701009387C70B94
:1044B00003A70700630A070083A6070003A74605B2
:1044C0001307170023AAE60403A50700678000006E
:1044D000130101FD2320210323261102232481023D
:1044E00023229102232E3101130905007370043039
:1044F00097C401009384840583A7040017C40100B6
:1045000013048406639E070A8327040083A7870594
:10451000639A0700832704001307100023AEE70403
:10452000639A050E83A704006388070083270400AD
:1045300083A74704639A07147370043083A70400A9
:10454000639407068327040003A587056308050015
:10455000630209048327040023AC070483270400B3
:1045600023AE070483A704006388070083270400A1
:1045700083A74704639207068320C10203248102B4
:1045800083244102032901028329C101130101038C
:104590006780000003270400832787059387F7FFC0
:1045A000232CF7046FF09FFB0327040083270400EC
:1045B00083274704938717002322F7046FF09FF89F
:1045C00003270400832704008327470493871700E9
:1045D0002322F7046FF05FF303270400832604000F
:1045E000832747049387F7FF2322F70483A7460412
:1045F000E39407F8736004308320C102032481022E
:1046000083244102032901028329C101130101030B
:1046100067800000032504002326B1001305450030
:10462000EFC08F9B8325C1009307F0FF6380F508DF
:1046300097C70100938707F283A9070003270400A7
:1046400083A70700B389B9002322370163ECF90679
:1046500097C70100938707F103A50700832504008E
:1046600093854500EFC00F9297C701009387C7EC71
:1046700083A7070063F6F90097C7010023AE37EB65
:10468000EFB01FF16FF01FEA032704008326040038
:10469000832747049387F7FF2322F70483A7460461
:1046A000E39C07E8736004306FF01FE98325040082
:1046B00017C501001305450E93854500EFC08F898E
:1046C0006FF01FFC97C70100938787E903A50700D8
:1046D0008325040093854500EFC0CF8A6FF05FFA11
:1046E000130101FD23202103232E31012326110272
:1046F0002324810223229102232C410113890500E6
:10470000930906007370043097C40100938404E495
:1047100083A7040017C40100130404E5639C071475
:1047200003270400930720000327C7056304F7024B
:10473000832704001345F5FF03A787053375E500BC
:1047400023ACA704832704001307100023AEE7045B
:10475000639A060A83A7040063880700832704007E
:1047600083A74704639407167370043083A704007B
:10477000639E0706638809008327040083A78705D3
:1047800023A0F9000327040093071000130500007D
:104790000327C705630EF700832704001349F9FFB9
:1047A0001305100003A787053379E90023AC27051B
:1047B0008327040023AE070483A70400638807004F
:1047C0008327040083A747046392070C8320C10258
:1047D0000324810283244102032901028329C101A8
:1047E000032A8101130101036780000003270400ED
:1047F0008327040083274704938717002322F704A5
:104800006FF05FF7032504002326D1001305450050
:10481000EFB09FFC8326C1009307F0FF638AF60C7C
:1048200097C70100938707D303AA07000327040053
:1048300083A70700330ADA00232247016368FA0CD2
:1048400097C70100938707D203A5070083250400BB
:1048500093854500EFB01FF397C701009387C7CD3D
:1048600083A707006370FA0A97C7010023A647CD04
:104870006F004009032704008327040083274704AF
:10488000938717002322F7046FF09FE903270400A2
:1048900083260400832747049387F7FF2322F70426
:1048A00083A74604E39407F2736004308320C102B7
:1048B0000324810283244102032901028329C101C7
:1048C000032A81011301010367800000032704000C
:1048D00083260400832747049387F7FF2322F704E6
:1048E00083A74604E39207E8736004306FF0DFE7C4
:1048F0008325040017C50100130505EA93854500CB
:10490000EFB05FE5EFB0DFC86FF0DFE497C70100FD
:10491000938707C503A507008325040093854500F9
:10492000EFB05FE66FF01FFE630A050C130101FF95
:10493000232611002324810023229100232021011A
:104940007370043097C40100938444C083A70400AB
:1049500063960708638606008327850523A0F60073
:1049600093070600930620000326C505232ED504D1
:1049700013870500130405006382D70A63F4F60861
:10498000930530006388B700930540006396B70035
:10499000630CD610232CE40493071000630CF60874
:1049A0001304100083A70400638C070097C701005D
:1049B000938787BB83A7070083A7470463980706ED
:1049C000130504008320C1000324810083244100D7
:1049D00003290100130101016780000097C701004E
:1049E000938787B803A7070083A707008327470497
:1049F000938717002322F7046FF0DFF573700430FC
:104A00006F00000093061000E398D7F88327850510
:104A100033E7B700232CE5046FF01FF883278505E3
:104A200093871700232CF5046FF01FF7EF40004722
:104A30006FF01FF91309440013050900EFB0DFD927
:104A400097C701009387C7B00325C40283A7070057
:104A500063F6A70097C7010023ACA7AE93054001FA
:104A6000EF40C02D97C70100938787C13385A7000A
:104A700093050900EFB01FCE8327840263860700E9
:104A8000737004306F00000097C701009387C7ADB3
:104A900083A707000327C40283A7C702E3F2E7F056
:104AA000EFB01FAF6FF0DFEF130400006FF09FEF68
:104AB00063080508130101FE232C8100232A9100BD
:104AC00023282101232631012324410123225101DE
:104AD000232E110093090700138A06009304060091
:104AE0001389050013040500EFB0DFBE930A05002B
:104AF00063060A00832784052320FA000327C405E0
:104B000093072000232EF4046380F40463FA9710C3
:104B1000930630006388D400930640006396D40067
:104B2000630CF70E232C2405930710006312F70A79
:104B30008327840263820702737004306F000000D1
:104B4000737004306F00000083278405938717007B
:104B5000232CF4046FF05FFD97C701009387879DB6
:104B600083A707006390070A930444001385040099
:104B7000EFB09FC697C701009387879D0325C402A6
:104B800083A7070063F6A70097C7010023A2A79C8D
:104B900093054001EF40801A97C70100938747AE05
:104BA000938504003385A700EFB0DFBA97C70100F3
:104BB0009387879B83A707000327C40283A7C702A5
:104BC00063F8E700638609009307100023A0F9004B
:104BD0001304100013850A00EFB05FAF1305040043
:104BE0008320C101032481018324410103290101A0
:104BF0008329C100032A8100832A41001301010295
:104C0000678000009305840117C50100130545B6B0
:104C1000EFB05FB46FF09FF9130400006FF09FFBDB
:104C200093071000E392F4F08327840533E927010A
:104C3000232C24056FF05FEF630A050E130101FEBC
:104C4000232C8100232A910013040500232631011F
:104C5000232E11002328210193840500EFB09FA784
:104C6000930720008326C405232EF404832784059C
:104C7000130710009309050093871700232CF404F1
:104C80006396E60883278402638607007370043006
:104C90006F00000097C701009387C78983A70700AB
:104CA000639A07081309440013050900EFB0DFB247
:104CB00097C701009387C7890325C40283A707000C
:104CC00063F6A70097C7010023A4A78893054001B6
:104CD000EF40C00697C701009387879A93050900A4
:104CE0003385A700EFB01FA797C701009387C78739
:104CF00083A707000327C40283A7C70263F8E7005E
:104D0000638604009307100023A0F40003248101AC
:104D10008320C10183244101032901011385090076
:104D20008329C100130101026FB05F9A73700430D0
:104D30006F0000009305840117C50100130545A30A
:104D4000EFB05FA16FF05FFA9307050063080506F7
:104D50007370043017B701001307477F83260700DD
:104D6000639E060203A6C7059306200013050000F4
:104D70006316D60023AE070413051000832707002F
:104D8000638C070097B701009387077E03A707008E
:104D900003274704631C07026780000097B60100E1
:104DA0009386867C03A6060083A606008326460417
:104DB000938616002322D6046FF0DFFA97B701001E
:104DC0009387877A83A707006FF09FF803A70700F0
:104DD00083A60700832747049387F7FF2322F7045E
:104DE00083A74604E39A07FA7360043067800000E3
:104DF000130101FB23229104232E3103232C4103B1
:104E0000232A510323286103232671032326110437
:104E100023248104232021052324810323229103B9
:104E20002320A10397B901009389097517BB0100DD
:104E3000130BCB7397B401009384847397BA01006A
:104E4000938A4A73130A1000930B900083A70900FA
:104E500003A707006304071883A7C70003A9070077
:104E6000EFD09FCEEFD0DFCF83270B00130C0500D0
:104E70006366F50E97B7010023AAA76E130600001C
:104E80006374252503A50400B3058941EFC05FCBFA
:104E9000EFD01FFF6304051803A50400930600006C
:104EA0001306000093050100EFC0CFC9E30005FA27
:104EB000832701000324810063D007028327410078
:104EC0008325C10013050400E78007008327010044
:104ED000E3C407FC032481008327440163860700A1
:104EE00013054400EFB05F8FEFD09FC783270B00FF
:104EF000130C05006362F50C8327010017B701004E
:104F000023268767E3EAFBF8B317FA0013F70721B4
:104F10006316072E13F7770C6316072693F707021D
:104F2000E38C07F613050400EF00D05C6FF0DFF6AA
:104F300083A7C70003A4C70083AC0700130944007C
:104F400013050900EFB05F898327440213050400AD
:104F5000E78007008327C4016386470D83A7090004
:104F600003A70700E31607FC03A70A0097B6010092
:104F700023AE865F97B6010023AEF65E97B70100B9
:104F800023ACE75EEFD0DFEF6FF01FF183A7C70020
:104F900003A9C70003AD0700930C490013850C005B
:104FA000EFB09F838327490213050900E7800700BC
:104FB0008327C901638C470B83A7090003A7070058
:104FC000E31607FC03A70A0097B6010023A4F65ACC
:104FD00097B7010023A2E75A6FF01FF2EFD0DFB6B8
:104FE000EFD01FB883270B00130C0500E368F5F61C
:104FF00083A70A0003A504001309000003A6070005
:10500000B305894117B701002322875713361600CD
:10501000EFC01FB3EFD0DFE6E31005E8EFB04FD7E6
:105020006FF09FE78327840193050900B387FC0095
:1050300063E2FC0883A704006386070223280100BB
:10504000232A9101232C8100EFF0CF9B03A50400BC
:10505000930600001306000093050101EFB01FAF97
:10506000E31E05EE737004306F0000008327890192
:1050700093850C00B307FD006362FD0883A704005D
:105080006386070223280100232AA101232C210182
:10509000EFF04F9703A504009306000013060000ED
:1050A00093050101EFB09FAAE31805F07370043077
:1050B0006F00000003A509002322F40023288400C8
:1050C000EFB04FEC6FF09FE9EFD09FDB83A70900B3
:1050D00083A7C70003A4C700930C440013850C00EA
:1050E000EFB08FEF8327C401638447038327440213
:1050F00013050400E78007006FF01FDA03A509001D
:105100002322F90023282901EFB0CFE76FF0DFEA6F
:1051100083278401232884003307F9002322E40035
:10512000636AEC04330C2C41636EFC0283A7040019
:105130006386070223280100232A2101232C8100F2
:10514000EFF04F8C03A50400930600001306000047
:1051500093050101EFB09F9FE31A05F873700430C7
:105160006F00000003A50A0093850C00EFB08FE1EB
:105170006FF0DFF703A5090093850C00EFB08FE017
:105180006FF0DFF683274100832684012328840003
:105190003387D7002322E400636AEC0AB307FC409C
:1051A00063EED7088327440213050400E780070055
:1051B0008327C401E39247CF8326840183274100DC
:1051C00003A70400B387D700630607022328010062
:1051D000232AF100232C8100EFF0CF8203A50400E5
:1051E000930600001306000093050101EFB01F961F
:1051F000E31405CA737004306F0000008327410078
:10520000232CF40063880702B38787012322F4006C
:1052100023288400930544006368FC0003A50A006A
:10522000EFB04FD66FF05FC703A50900EFB08FD581
:105230006FF09FC6737004306F00000003A50A0072
:1052400093054400EFB00FD46FF01FC56374FC00EA
:10525000E37AF7F403A5090093054400EFB08FD279
:105260006FF09FC3130101FF232481002326110047
:10527000232291002320210117B401001304442F9D
:10528000EFF00F988327040063840704EFF08F9AF0
:1052900083270400638A07029308000013080000B4
:1052A0009307000013072000930600001306004038
:1052B00097B501009385851017050000130585B388
:1052C000EFC05F9C63140506737004306F0000002C
:1052D00017B901001309894D13050900EFB00FC577
:1052E00097B401009384C44D13850400EFB00FC43C
:1052F00013060000930500011305400097B7010055
:1053000023AC272797B7010023A69726EFB0CFEF4E
:1053100017B70100232EA7246306050297B50100E5
:1053200093854509EFC08FEE6FF05FF68320C100D3
:10533000032481008324410003290100130101019A
:1053400067800000737004306F000000638A050AF4
:10535000130101FD232A5101930A05001305C00220
:10536000232481022322910223202103232E3101B1
:10537000232C4101232611022328610123267101D8
:105380001309070093890600130A06009384050099
:10539000EF00407E13040500630C0502EFF04F861A
:1053A00097B701009387C71C83A70700638E070484
:1053B000EFF04F881305440023205401232C940060
:1053C000232E44012320340323222403EFB00FB8FB
:1053D000130504008320C1020324810283244102B7
:1053E000032901028329C101032A8101832A410182
:1053F000032B0101832BC10013010103678000000F
:10540000737004306F00000097BB0100938B0B3A60
:1054100013850B00EFB08FB117BB0100130B4B3A94
:1054200013050B00EFB08FB01306000093050001C9
:105430001305400097B7010023A0771597B7010027
:1054400023AA6713EFB04FDC17B701002322A7127E
:10545000630A050097B501009385C5F5EFC00FDB22
:105460006FF01FF5737004306F000000630E0506C7
:10547000130101FE232C8100232E1100232A910009
:1054800017B401001304C40E832804001308050098
:105490001305000063800804930407002320B10073
:1054A000138706002322C100232401019306500024
:1054B00063C0B604EFE01FD593072000630EF50428
:1054C0000325040093060000130600009305010065
:1054D000EFB0CFE78320C101032481018324410180
:1054E0001301010267800000737004306F00000038
:1054F00093050100930600001306070013850800BA
:10550000EFB09FB68320C1010324810183244101B0
:1055100013010102678000000325040093060000C8
:105520001386040093050100EFB04FE26FF09FFA7D
:1055300063060500032505006780000073700430D2
:105540006F00000063160500737004306F000000E8
:10555000130101FF232611002324810013040500F9
:10556000EFE01FEA032544013334A000EFE09FEC95
:10557000130504008320C1000324810013010101ED
:105580006780000063160500737004306F00000030
:10559000130101FF232481001304050023261100B9
:1055A000EFE01FE603240402EFE0DFE88320C10000
:1055B000130504000324810013010101678000002A
:1055C00063160500737004306F000000130101FFC3
:1055D00023248100232291001384050093040500F5
:1055E00023261100EFE0DFE123A0840203248100E1
:1055F0008320C10083244100130101016FE09FE378
:10560000130101FE232E110097B70100938747F67F
:105610002322A10003A50700938706002324B100DD
:105620002326C1009305010013860700930600009E
:105630009307E0FF2320F100EFB01FA38320C101F7
:10564000130101026780000097B70100938747F2BA
:1056500083A8070063960800737004306F00000091
:10566000130101FE930706001387050013080500C8
:1056700013860600930501001385080093060000B9
:105680009308F0FF232E1100232011012322010192
:105690002324E1002326F100EFB04FCB8320C1018A
:1056A0001301010267800000630C0500B70700FFCB
:1056B000B3F7F500638A0700737004306F000000D1
:1056C000737004306F000000130101FF2324810078
:1056D0002322910023261100130405009384050062
:1056E000EFE01FD20327040093C7F4FFB377F7005E
:1056F0002320F400032481008320C100832441007F
:10570000130101016FE01FD3630C0500370700FF91
:10571000B3F7E500638A0700737004306F00000080
:10572000737004306F0000006F30007A130101FFC6
:105730001305C0012324810023261100EF008043BC
:105740001304050063080500232005001305450028
:10575000EFA0DFFD130504008320C10003248100B6
:10576000130101016780000063020502B70700FF13
:10577000B3F7F50063860700737004306F00000014
:10578000639A0500737004306F000000737004307A
:105790006F000000130101FE232C8100232821014A
:1057A000232631012324410123225101232E1100FC
:1057B000232A91009309070013890600930A060023
:1057C00013840500130A0500EFE0DFA3631805004A
:1057D00063860900737004306F000000EFD0CFB60D
:1057E00083240A00B37794006312090463820704D8
:1057F00063880A009347F4FFB3F797002320FA0069
:10580000EFD00FE88320C101032481011385040038
:1058100003290101832441018329C100032A810056
:10582000832A41001301010267800000E302F4FCB7
:10583000E38809FCB335500193958501630609009F
:10584000B7070004B3E5F50013860900B3E585004A
:1058500013054A00EFE04FCDEFD08FE2631405004F
:10586000EFA01FD3EFE09FC19317650093090500D8
:1058700063DA0700B70400019384F4FFB3F49900DE
:105880006FF05FF8EFE0DFB783290A00B3773401E8
:1058900063100902638A070063880A009347F4FFD4
:1058A000B3F737012320FA00EFE0DFB86FF09FFC79
:1058B000E31CF4FE6FF05FFE630C0500B70700FF0A
:1058C000B3F7F500638A0700737004306F000000BF
:1058D000737004306F000000130101FF2324810066
:1058E0001304050023261100232291002320210107
:1058F00013890500EFE0DFB0832404009345F9FF2E
:10590000B3F795002320F400EFE0DFB28320C1005D
:10591000032481001385040003290100832441002E
:105920001301010167800000138605009306000043
:105930009305050017050000130545D76FF05FCCF0
:10594000130101FF23248100130405002326110005
:10595000EFA05FD803240400EFA05FD78320C1002D
:105960001305040003248100130101016780000076
:10597000630C0500370700FFB3F7E500638A0700F3
:10598000737004306F000000737004306F0000000B
:105990006F308053B70700FFB377F60063860700C8
:1059A000737004306F0000006316060073700430DB
:1059B0006F000000130101FE232C81002328210128
:1059C0002326310123244101232E1100232A910093
:1059D0001389060093890500130A050013040600C5
:1059E000EFE05F82631E05046306090073700430F4
:1059F0006F000000EFD04F9583240A0093850900C3
:105A000013050A00B3E49900EFF09FF6B377940012
:105A1000630AF40883240A00EFD08FC68320C101F3
:105A2000032481011385040003290101832441011A
:105A30008329C100032A810013010102678000004D
:105A4000EFD08F9083240A009385090013050A0084
:105A5000B3E43401EFF0DFF1B3F78400638487042B
:105A6000E30A09FAB705000513060900B365B40097
:105A700013054A00EFE04FABEFD08FC06314050071
:105A8000EFA01FB1EFE09F9F9317650093040500FF
:105A900063D40702B70700019387F7FFB3F4F4005C
:105AA0006FF0DFF783270A001344F4FFB3F7870092
:105AB0002320FA006FF05FF6EFE09F9483240A0042
:105AC000B3779400639887009347F4FFB3F7970088
:105AD0002320FA00EFE01F966FF0DFFB130101FFB8
:105AE00023248100232611001304050023229100A2
:105AF000EFD08F85832744006386070203250401C6
:105B00009304C400631895006F008003032504010B
:105B100063089502B7050002EFE04FCB83274400EE
:105B2000E39607FE13050400EF00C01C0324810068
:105B30008320C10083244100130101016FD04FB4C1
:105B4000737004306F000000930606001386050092
:105B50009305050017050000130545BB6FF05FAA0C
:105B6000630605000325850167800000130500001A
:105B700067800000130101FF232481002326110008
:105B800013040500EFC05FFC97B701009387079FE0
:105B900083A70700639C0704B797010017B70100AC
:105BA000130787C39387C7FF97B6010023AEE69C10
:105BB00017B701002328F79C17B701002320F7C26D
:105BC00097B701009387C79B17B701002326F7C03B
:105BD0009307100017B70100232A079A17B701008F
:105BE0002320079A17B70100232AF79863120402AB
:105BF000EFD00FA9EF10C0601304000013050400DC
:105C00008320C1000324810013010101678000008B
:105C100013058400937735006398070CB79701004C
:105C20001307F5FF9387A7FFE3E4E7FC97B60100AE
:105C30009386869583A706006F00400103A707009F
:105C4000630A0700938607009307070003A747002E
:105C5000E366A7FE17B7010013078792E38AE7F808
:105C600003A70700130600011384870023A0E600A2
:105C700003A74700B306A740637ED6023388A70078
:105C80002322D80023A2A7008325480097B601004D
:105C90009386868F6F0080009306070003A7060097
:105CA00003264700E36AB6FE2320E80023A006018E
:105CB00003A7470097B701009387479183A7070081
:105CC000B387E74017B701002322F790EFD04F9B2F
:105CD000E30204F2130504008320C10003248100C1
:105CE00013010101678000001375C5FF130545000E
:105CF0006FF0DFF263080506130101FF2324810022
:105D00002326110013040500EFC01FE4930584FF50
:105D10000326C4FF17B70100130707876F00800031
:105D2000138707008327070083A64700E3EAC6FE20
:105D3000232CF4FE2320B70097B70100938707892F
:105D400003A707008327C4FF032481008320C10029
:105D5000B387E70017B70100232AF7861301010173
:105D60006FD00F926780000097B701009387078676
:105D700003A5070067800000678000003367B50057
:105D80001377370093070500631207049308D6FFC3
:105D9000B308150113070500938605006378150302
:105DA00003A806001307470093864600232E07FF2B
:105DB000E36817FF9347F5FFB387170193F7C7FF12
:105DC00093874700B385F500B307F5003306C50098
:105DD00063F4C70C9386450013884700B3B6D70019
:105DE00033B8050133E7F50093C6160013481800D1
:105DF00013773700B3E60601133717003377D70060
:105E0000330EF64093861700630807061337AE007B
:105E10006314070613532E001388050093860700AA
:105E20001307000083280800130717001308480011
:105E300023A0160193864600E36667FE1377CEFF24
:105E4000B385E500B387E7006306EE0483C605006B
:105E5000138717002380D700637EC70283C615000F
:105E600013872700A380D7006376C70203C72500E6
:105E70002381E70067800000B307F640B387F50091
:105E80009385150003C7F5FF93861600238FE6FE62
:105E9000E398F5FE6780000067800000B367C500E7
:105EA00093F73700B308C5006382070E63761511B8
:105EB000B307A04093F737001387370093065000CD
:105EC00093F5F50F130815003383A8401306F6FF6A
:105ED0006374D700130750006368E60E6380070EF3
:105EE0002300B50013071000638EE700A300B50080
:105EF00013073000130825006396E70013083500E8
:105F00002301B5001396850033E6C50013970501FC
:105F10003367E6003303F34093968501B366D700F9
:105F200013562300B307F5001307000023A0D70082
:105F30001307170093874700E36AC7FE1377C3FF71
:105F4000B307E8006300E3082380B7001387170056
:105F5000637C1703A380B7001387270063761703BA
:105F60002381B7001387370063701703A381B7003D
:105F700013874700637A17012382B70013875700FE
:105F800063741701A382B7006780000093F5F50FD3
:105F900013978500B365B700139705013367B70002
:105FA000E37415FF930705009387470023AEE7FED0
:105FB000E3EC17FF6780000067800000130805000E
:105FC0006FF05FF467800000930705006FF0DFF764
:105FD0008347050013070500638C070013051500B0
:105FE00083470500E39C07FE3305E540678000001A
:105FF0001305000067800000130515008347F5FFB7
:106000009385150003C7F5FF63880700E386E7FE65
:106010003385E74067800000930700006FF05FFF63
:10602000930705009385150003C7F5FF93871700B5
:10603000A38FE7FEE31807FE678000008346050094
:10604000930700026398F6001305150083460500C8
:10605000E38CF6FE938756FD93F7D70F6380070412
:1060600093070500930500006388060413050000EC
:1060700093871700138606FD1317250083C60700B4
:106080003305A700131515003305A600E39206FE9D
:10609000638405003305A04067800000938536FDCA
:1060A0008346150093B5150093071500E39006FC91
:1060B000130500006FF0DFFD13050000678000008E
:1060C00083A705002380A70083A7050093871700F7
:1060D00023A0F5006780000097A601009386464B39
:1060E00083A70600173703001307C771138617002D
:1060F000B307F7002380A70097A5010023AAC5488E
:106100009307A000630AF500930700046308F600F4
:106110001305000067800000E30C06FE370610F050
:10612000130717008347F7FF2320F6F083A7060025
:106130009387F7FF97A5010023ACF544E39207FE90
:106140001305000067800000130101EB2322911466
:1061500023202115232A51132324811323261114CC
:1061600023248114232E3113232C4113232861135C
:1061700023267113232291132320A113232EB1115F
:1061800093040500138905002326C100130C500257
:10619000930A90008347090063888703638C07068E
:1061A00003A404006F008000638607062300F40048
:1061B00003A40400130919001304140023A084008D
:1061C00083470900E39287FF0346190093081900EB
:1061D00093860800130D00029309F0FF130AF0FFE5
:1061E00013080000130550059307D6FD93F7F70F2A
:1061F00013891600636EF53A17A70100130787E0AD
:1062000093972700B387E70083A70700B387E700CA
:10621000678007008320C114032481148324411460
:10622000032901148329C113032A8113832A4113EB
:10623000032B0113832BC112032C8112832C4112D7
:10624000032D0112832DC111130101156780000078
:10625000930C8000232401009307100063DA071DCC
:106260008327C10003A40400938B770093F68BFF70
:1062700003AB060083A94600938786002326F1001E
:1062800013860C009306000013050B00938509008C
:10629000EF20C05A2328A100930700006380373302
:1062A000930D4101930B100013860C009306000020
:1062B00013050B0093850900EF10907A93060000F8
:1062C00013860C00130B050093890500EF2000577F
:1062D0008327810023A0AD0093861B00938D4D0082
:1062E00063863701938B06006FF01FFCE37C9BFFF6
:1062F00063D24603930704002380A70103A404008C
:10630000130AFAFF9307140023A0F4001384070074
:10631000E3C446FF93962B0093070101B386D70091
:106320006F008002938777052300F40003A4040024
:10633000938BFBFF93871B001304140023A084009E
:106340009386C6FFE358F0E483A70600E3ECFAFC6B
:10635000938707036FF05FFD83A704009306000394
:106360000327C1002380D70083A7040093064700BA
:10637000930C00011386170023A0C40013068007A6
:10638000A380C70003A4040023240100930707008F
:106390001304140023A0840003AB0700930900003A
:1063A0002326D1006FF0DFED8327C10083AC070007
:1063B000938B470063880C28635C40259307D002C9
:1063C000631EFD2083C70C006388070263D809247D
:1063D00083A60400938C1C00130AFAFF2380F600A6
:1063E00003A404001304140023A0840083C70C003A
:1063F000E39E07FC6352400303A4040093070002DA
:106400002300F40003A40400130AFAFF1304140089
:1064100023A08400E3160AFE232671016FF09FD7A4
:106420002324010093071000930CA000E3CA07E3A4
:106430008327C10003A40400938647006FF0DFF5B3
:1064400003C61600930609006FF01FDA83A7040045
:10645000930650022380D70003A404001304140001
:1064600023A084006FF01FD3930C000123240100AC
:106470006FF09FDE8327C10003C616009306090054
:1064800083A90700938747002326F100E35E0AD41F
:10649000138A09009309F0FF6FF01FD503C6160099
:1064A000130DD002930609006FF01FD49347FAFF33
:1064B00093D7F74103C61600337AFA009306090012
:1064C0006FF09FD203C61600130D00039306090058
:1064D0006FF09FD183C51600930906FD930609004E
:1064E000938705FD13860500E3E2FAFA93972900E6
:1064F000B38937019386160093991900B389B900BF
:1065000083C50600938909FD938705FD1386050061
:10651000E3FEFAFC6FF09FF70327C10083A7040096
:1065200083260700130747002326E1002380D700B6
:1065300003A404001304140023A084006FF09FC57B
:106540009307100063D4070F8327C1009386770059
:1065500093F686FF938786002326F10083A94600E1
:1065600083A7060063DE090E83A604001306D0028B
:10657000B307F0402380C60003A40400B336F00044
:10658000B30930411304140023A08400138B0700C7
:10659000B389D940930CA000232401006FF05FCE93
:1065A00003C6160013081800930609006FF0DFC336
:1065B00083A70400138908006FF09FE9E3729BCF63
:1065C00093071000930B000093061000E3C447D319
:1065D0006FF05FD497AC0100938CCCDE93850900FB
:1065E00013850C00EF100070330AAA406352400379
:1065F00003A404002300A40103A40400130AFAFF67
:106600001304140023A08400E3160AFE130A0000FA
:1066100083C70C00E38207E0E3CC09DA9389F9FF32
:106620001307F0FFE396E9DA6FF0DFDC8327C100A0
:106630009386470083A707002326D10093D9F7410B
:106640006FF05FF2635640019307D002E314FDF848
:1066500097AC0100938C0CD7930780026FF01FD783
:10666000138B0700930CA0002324010003A4040053
:106670006FF01FC1130101EB232E3113B709004046
:106680009387F9FF2324811423229114232C41138F
:10669000232A5113232611142320211523286113A3
:1066A0002326711323248113232291132320A11362
:1066B000232EB111130A05002324B10017A40100F1
:1066C000130404ED973A0300938ACA1397A40100B8
:1066D0009384C4A82326F100930550021305A0005B
:1066E00013080004B70610F083470A00638EB7044E
:1066F0006388070A03270400130A1A001306170009
:106700003387EA0097A8010023A4C8E82300F70014
:106710006380A708E31A06FD173703001307870EE7
:10672000130717008347F7FF23A0F6F08327040021
:106730009387F7FF17A60100232CF6E4E39207FEE8
:1067400083470A00E396B7FA83461A0013051A0036
:1067500013070500930B0002130BF0FF130CF0FF5F
:106760001308000093055005930890009387D6FD09
:1067700093F7F70F130A170063ECF544939727007C
:10678000B387970083A70700B38797006780070048
:106790001737030013070707E31406F86FF0DFF459
:1067A0008320C11403248114832441140329011478
:1067B0008329C113032A8113832A4113032B011355
:1067C000832BC112032C8112832C4112032D011241
:1067D000832DC1111301011567800000930C800007
:1067E000130D00009307100063DA0721832781004F
:1067F0009387770093F787FF83AD070003AB4700CC
:10680000138787002324E10013860C009306000001
:1068100013850D0093050B00EF2040022328A100F3
:1068200063086D45130941019309100013860C009C
:106830009306000013850D0093050B00EF10502206
:1068400013860C0093060000930D0500138B0500C2
:10685000EF10D07E2320A900938919001309490065
:10686000E3166DFDE3F49DFD13060004B70610F07A
:1068700063D489038327040013871700B387FA00C2
:1068800097A5010023A6E5D023807701630AC706F8
:10689000130CFCFFE3C089FF8327C1001305C1006F
:1068A00093089000B386F9009396260093070101A0
:1068B000B386D7001308A00013030004370610F0B6
:1068C000E38CA6E083A706009305000363F4F800B9
:1068D0009305700503270400B387B70093051700DD
:1068E0003387EA0017AE01002324BECA2300F70055
:1068F00063860737638C65329386C6FF6FF05FFC53
:1069000017370300130707F0130717008347F7FF34
:1069100023A0F6F0832704009387F7FF97A50100D3
:1069200023A8F5C6E39207FE130CFCFF6FF09FF659
:1069300083270400130600041387170097A501009E
:1069400023A8E5C4B386FA00930500032380B600AC
:106950006308C7509387270097A6010023AAF6C2B1
:106960003387EA00930680072300D7001737030018
:10697000130747E9B70610F06392C7021307170021
:106980008347F7FF23A0F6F0832704009387F7FFE0
:1069900017A60100232EF6BEE39207FE832781008F
:1069A000930C0001130D000093874700032781001B
:1069B000130B0000832D07002324F1006FF0DFE4A8
:1069C0008327810083AC070013894700638E0C4C3A
:1069D0006358802B9307D0026394FB3E03C70C00DF
:1069E000930507006314072A6F00002F9307100018
:1069F000930CA000130D0000E3CA07DF832781007A
:106A0000938747006FF09FFA832781008346170022
:106A100013070A0003AB0700938747002324F10004
:106A2000E3560CD4130C0B00130BF0FF6FF01FD4C4
:106A300083461700930BD00213070A006FF01FD391
:106A40009347FCFF93D7F74183461700337CFC0044
:106A500013070A006FF09FD183461700930B0003C2
:106A600013070A006FF09FD003461700138B06FD33
:106A700013070A00930706FD93060600E3E2F8FAFF
:106A800093172B00B387670113071700939717001D
:106A9000B387C70003460700138B07FD930706FD66
:106AA00093060600E3FEF8FC6FF09FF78325810054
:106AB000832704001306A00003A705009386170090
:106AC000B387FA0017A501002324D5AC2380E70083
:106AD000138945006300C736930700046384F62AD0
:106AE000232421016FF05FBF9307100063DE073599
:106AF0008327810013877700137787FF9307870029
:106B00002324F100032B47008327070063560B3E25
:106B100003270400130600049306170097A501003D
:106B200023A8D5A63387EA009305D0022300B70037
:106B3000638CC638B307F0403337F000330B604145
:106B4000938D0700330BEB40930CA000130D000056
:106B50006FF09FCB834617001308180013070A0035
:106B60006FF0DFC08346170013070A006FF01FC0E5
:106B700083270400930600041387170017A601005B
:106B80002328E6A0B387FA00130650022380C7002B
:106B9000E314D7B4173703001307C7C6B70610F0BE
:106BA000130717008347F7FF23A0F6F0832704009D
:106BB0009387F7FF17A60100232CF69CE39207FEAC
:106BC0006FF09FB1930C0001130D00006FF09FC197
:106BD0008327040093060004130A05001387170097
:106BE00017A601002326E69AB387FA00130650027F
:106BF0002380C700E312D7AE17370300130787C0FF
:106C0000B70610F0130717008347F7FF23A0F6F02D
:106C1000832704009387F7FF17A60100232AF6961F
:106C2000E39207FE130A05006FF01FAB173703004E
:106C3000130747BD130717008347F7FF2320F6F01C
:106C4000832704009387F7FF97A5010023A2F594FB
:106C5000E39207FE9386C6FF6FF09FC617370300C7
:106C6000130747BAE39805FC9386C6FF6FF05FC52C
:106C7000E3FA9DBB930910006FF01FBF130C0000D7
:106C800003C70C0093050700E30C07E49308F0FF2B
:106C90001305A00013080004B70610F0635E0B0C88
:106CA0008327040013861700B387FA0017A3010097
:106CB0002320C38E2380E7006382A5086308060BA8
:106CC000938C1C0003C70C00130CFCFF93050700FA
:106CD000E31607FCE35680E18327040093050002D6
:106CE00013060004B70610F06F00C000130CFCFF81
:106CF000E3080CDE13871700B387FA002380B70080
:106D000017A501002326E58893070700E310C7FEB7
:106D100017370300130707AF130717008347F7FF61
:106D200023A0F6F0832704009387F7FF17A501003F
:106D30002320F586E39207FE6FF05FFB1737030011
:106D4000130747ACE30E06F6130717008347F7FF58
:106D500023A0F6F0832704009387F7FF17A601000E
:106D60002328F682E39207FE6FF09FF517370300A2
:106D7000130747A96FF05FFD130BFBFFE3121BF333
:106D80006FF05FF5173703001307C7A7B70610F0BA
:106D9000130717008347F7FF23A0F6F083270400AB
:106DA0009387F7FF179601002324F67EE39207FEF0
:106DB000232421016FF05F92979C0100938C8C60DB
:106DC00093050B0013850C00EF00D071330CAC4021
:106DD000E35880EB8327040013060004B70610F085
:106DE0006F00C000130CFCFFE30A0CE813871700C8
:106DF000B387FA00238077019795010023AAE578ED
:106E000093070700E310C7FE173703001307879F98
:106E1000130717008347F7FF23A0F6F0832704002A
:106E20009387F7FF9795010023A4F576E39207FE79
:106E30006FF05FFB173703001307C79CE39806F456
:106E4000232421016FF05F89832781001387470086
:106E500083A707002324E10013DBF7416FF01FCB6A
:106E6000173703001307079AB70610F01307170028
:106E70008347F7FF23A0F6F0832704009387F7FFEB
:106E8000179601002326F670E39207FE9307100081
:106E900017970100232EF76E93078007173703001B
:106EA0002302F7966FF09FAF635680019307D002DD
:106EB000E394FBF0979C0100938CCC501307800265
:106EC000930580026FF09FDC9736030093868693CC
:106ED000370610F09386160003C7F6FF2320E6F06E
:106EE000032704001307F7FF9795010023A2E56A23
:106EF000E31207FE6FF01FC4938D0700930CA000F0
:106F0000130D00006FF05F90B70710F023A0A7F2F9
:106F10006F000000130101FC130341022322B102A0
:106F200093050300232E11002324C1022326D1023E
:106F30002328E102232AF102232C0103232E11032B
:106F400023266100EFF00FF38320C1011305000039
:106F50001301010467800000130101FB1303810387
:106F6000232481022326A100232CC102130405003F
:106F7000130603001305C100232611022322F10486
:106F8000232ED1022320E104232401052326110509
:106F9000232E6100EFF04F9B8327C1002380070061
:106FA0000325C1008320C1023305854003248102EB
:106FB0001301010567800000B70710F083A647F4AE
:106FC00003A607F403A747F4E31AD7FEB716000099
:106FD000938606FAB306D60033B6C600B305E600BC
:106FE00023A4D7F423A6B7F467800000B70710F0F6
:106FF00003A747F403A607F483A647F4E31AD7FED2
:10700000B7160000938606FAB306D60033B6C6005C
:1070100023A4D7F4B305E60023A6B7F4930700082A
:1070200073A0473067800000130101FF2324810013
:1070300023261100130440011304F4FFEF00502F26
:10704000E31C04FE8320C10003248100130101011D
:1070500067800000130101FF232481002326110013
:1070600097970100938747531794010013048452A4
:1070700003A70700832704001306F07C9306470646
:10708000938747069795010023A8D550979501004F
:1070900023A2F550634AD6008320C1000324810057
:1070A00013010101678000001307478997970100CA
:1070B00023A4E74EEF00103A930710006316F50281
:1070C00003270400B71700009387F7761305000025
:1070D000E3D4E7FCEFF05FE3032481008320C100E9
:1070E000130101016FB05FA5179501001305052E6F
:1070F000EFF05FE213052000EFF01FE103248100B1
:107100008320C100130101016FB01FA31795010077
:107110001305452D6FF01FE0179501001305052D90
:107120006FF05FDF130101FF232481002322910010
:1071300023261100B7140000179401001304842BB8
:1071400093878438130000009387F7FFE39C07FEC2
:1071500013050400EFF01FDC6FF09FFE130101FF29
:107160002326110023248100EF00D00C1707000014
:107170001307C7EB930600001306100093052003C6
:107180001795010013058527EFE04F9C13040500B8
:10719000EFB01F9D130605001305040003248100B2
:1071A0008320C10013070000930600009305100020
:1071B000130101016FE08FAB130101FF23261100C2
:1071C000EF0050291307100093070000631AE50031
:1071D0008320C100138507001301010167800000AF
:1071E000179501001305851EEFF0DFD28320C10043
:1071F0009307200013850700130101016780000039
:10720000737004306F0000006780000073700430FA
:107210006F000000130101FF2322910023202101B0
:10722000232611002324810013090500EFC09FFCD1
:10723000979701009387073883A7070093045000AE
:107240006382A70A17940100130444371305000052
:10725000EFC04FFA032504001307F0FF9306000068
:107260001306100093850400EFE00FD0E31005FE35
:107270006F000004EFC00FF8032504009306F0FF31
:107280001306F00093050900EFE0CFF01375F50049
:107290001307F0FF93061000130600009305F0009B
:1072A000631A950403250400EFE00FCC6310050476
:1072B00013050000EFC00FF4032504009306F0FF50
:1072C0001306F00093050900EFE0CFEC9374F5008E
:1072D0009307F00013050000E38EF4F87370043098
:1072E0006F000000930430006FF0DFF5737004301E
:1072F0006F000000737004306F000000130101FE86
:10730000232C81002326310123244101232E110047
:10731000232A910023282101179401001304042A31
:10732000979901009389092A130AF00F13050000A9
:10733000EFC04FEC032504001307F0FF9306100085
:107340001306100093052000EFE00FC2130905009B
:10735000032504001307F0FF930610001306000036
:107360009305200AEFE04FC01375250A9307200A02
:10737000930410006308F51213050000EFC08FE7B7
:10738000032504001307F0FF9306100013061000F6
:107390009305200AEFE04FBD6304450193041000FC
:1073A00013050000EFC00FE5032504009306F0FF6E
:1073B0001306F00093052000EFE0CFDD1375F50014
:1073C0009307F0006304F500930410000325040004
:1073D00093050000EFE0CFD96302050A03250400FE
:1073E0009305000093041000EFE00FCD130500009B
:1073F000EFC04FE0032504009306F0FF1306F000F2
:1074000093052000EFE00FD91375F5009307F00006
:107410006304F500930410000325040093050000A5
:10742000EFE00FD563020502032504001307F0FF08
:1074300093061000130600009305F000EFE0CFB2B2
:10744000737004306F000000032504001307F0FF81
:1074500093061000130600009305F000EFE0CFB094
:10746000E31005FEE39E04FC83A709009387170041
:10747000179701002328F7146FF05FEB0325040032
:1074800093050000EFE04FC363140502639204020A
:1074900083A7090093871700179701002324F71289
:1074A0006FF0DFF49304E9F5B33490006FF0DFEC94
:1074B000930410006FF09FF3130101FD23202103BB
:1074C000232611022324810223229102232E31013B
:1074D000232C4101232A5101232861012326710114
:1074E00023248101232291012320A10113090500F6
:1074F000EFE0CFA39797010023A2A70C63020552E8
:10750000179A0100130A0A0B03250A009799010034
:107510009389090A13041000EFA0DFD69304050035
:1075200003A50900EFA01FD693073000630EF54EA8
:10753000930B8000930A1000979401009384040831
:10754000130B2000130C300003250A00EFB04F8A04
:1075500003A50900EFB0CF8903250A00EFA09FD251
:10756000630465011304100003A50900EFA09FD177
:10757000630465011304100003A5040093850A0049
:10758000EFE00FBF93F73A0003250A006398074422
:10759000EFA05FCF630465011304100093F75A0056
:1075A00003A5090063960742EFA0DFCD63046501E0
:1075B00013041000938BFBFF939A1A00E3960BF8C9
:1075C00003250A00179D0100130D0D00930A2000EA
:1075D000EFB00F8203A50900930B1000930C000A73
:1075E000EFB00F8103A50400130B3000130CD0057E
:1075F000EFE0CFCEEFE08F939797010023A0A7FC99
:10760000630C054013050900EFA09FFE1305090058
:10761000EFA05FC7630455011304100003A5040025
:107620009305200AEFE0CFB403A504001307000080
:1076300093060000130600009305F00FEFE0CF92D1
:10764000630495011304100013050900EFA09FC304
:10765000630455011304100003A504009305D00F23
:10766000EFE00FB103A5040013070000930600002C
:10767000130600009305F00FEFE00F8F9307D00F74
:107680006304F5001304100013050900EFA09FBF69
:10769000630455011304100003A5040093052000A2
:1076A000EFE00FAD13050900EFA0DFBD6304650136
:1076B0001304100003A5040093050000EFE04FAB96
:1076C0009307F00F6304F5001304100003A50400F2
:1076D00093052000EFE04F9E9307F00F6304F50041
:1076E0001304100013050900EFA09FF01305090013
:1076F000EFA05FB9630455011304100003A5040053
:1077000093052000EFE0CFA613050900EFA09FB777
:10771000630465011304100003A5040013070000AF
:1077200093060000130600009305F00FEFE0CF83EF
:10773000630485011304100003A504009305F00FF2
:10774000EFE08F97630485011304100003A5040084
:1077500093050000EFE04F9663040500130410004A
:1077600013050900EFA01FB26304650113041000A4
:1077700003250A00EFA01FB1630465011304100084
:1077800003A50900EFA01FB06304650113041000F6
:1077900003A504009305E000EFE08F9D03A504001E
:1077A0009306F0FF1306100093051000EFE08F9E84
:1077B00013751500631405001304100003A50400DD
:1077C00093050000EFE04F8F9307E0006304F5009E
:1077D0001304100003A504009305E000EFE0CF8D33
:1077E00003A5040093050000EFE00F8D630405007E
:1077F0001304100013050900EFA09FDF03250A0002
:10780000EFA01FDF03A50900EFA09FDE130509000D
:10781000EFA05FA7630455011304100003250A00BD
:10782000EFA05FA6630455011304100003A509002F
:10783000EFA05FA5630455011304100003A5040025
:107840009306F0FF1306F00093051000EFE08F940D
:107850001375F5009307F0006304F500130410009E
:1078600003A5040093050000EFE00F856304050005
:107870001304100013050900EFA0DFA063046501E5
:107880001304100003250A00EFA0DF9F63046501C5
:107890001304100003A50900EFA0DF9E6304650137
:1078A0001304100013050900EFA09FD403250A005C
:1078B000EFA01FD403A50900EFA09FD31305090073
:1078C000EFA05F9C630455011304100003250A0018
:1078D000EFA05F9B630455011304100003A509008A
:1078E000EFA05F9A63045501130410009305200074
:1078F00013050000EFA09FB503A504009306F0FF59
:107900001306F00093051000EFE0CF881375F50023
:107910009307F0006304F5001304100003A50400AE
:1079200093050000EFD05FF9630405001304100015
:1079300013050900EFA01F956304750113041000DF
:1079400003250A00EFA01F946304750113041000BF
:1079500003A50900EFA01F93630475011304100031
:107960001305000093050000EFA05FAE13050900AA
:10797000EFA05F91630455011304100003250A0072
:10798000EFA05F90630455011304100003A50900E4
:10799000EFA05F8F630455011304100003A50400DA
:1079A000EFE0CF9313050900EFA0DF8D63046501BD
:1079B0001304100003250A00EFA0DF8C63066503A3
:1079C00003A50900EFA01F8C737004306F00000046
:1079D000EFA05F8BE31E85BD6FF0DFBDEFA09F8A38
:1079E000E31C85BB6FF09FBB03A50900EFA09F8937
:1079F000E31C65FDE31A04FC83270D009387170041
:107A0000179701002322F7BCEFD05FD297970100B0
:107A100023A6A7BAE31805BE737004306F000000F8
:107A2000737004306F0000001384D4FF333480007F
:107A30006FF01FB0130101FE93080000130800004F
:107A40009307C100130710009306000013060040BF
:107A5000979501009385C59B170500001305458A7E
:107A6000232E1100EFA00FA28326C100930800006F
:107A700013080000930700001307000013060040DE
:107A8000979501009385459917050000130505A3F7
:107A9000EFA04F9F93080000130800009797010084
:107AA000938747B113071000930640001306004068
:107AB000979501009385C59617F5FFFF1305C575CA
:107AC000EFA04F9C97970100938787AE9308000023
:107AD00013080000130710009306800013060040EF
:107AE000979501009385C59317F5FFFF1305C572A0
:107AF000EFA04F9997970100938787AB83A7070063
:107B000063800702EFD09FC29797010023A6A7AA20
:107B1000630C05008320C10113010102678000008E
:107B2000737004306F000000737004306F00000049
:107B3000130101FF232611002324810097970100E0
:107B40009387C7A683A707001307400693871700EC
:107B50009796010023ACF6A46382E7021307800C1A
:107B6000638CE7081307C0126382E7048320C10017
:107B700003248100130101016780000017940100B4
:107B8000130484A303250400EFD09FDB63080504DE
:107B900093071000179701002328F7A08320C10046
:107BA0000324810013010101678000009797010001
:107BB000938787A003A5070093052001EFD0DFD6A8
:107BC00093071000630EF50417970100232EF79C0E
:107BD0009797010023AC079C6FF05FF90325040021
:107BE0001306000093052001EFD01FF69307100045
:107BF000E310F5FA6FF09FF7979701009387C79B03
:107C000003A50700EFD0DFD393072001E300F5F6CB
:107C100093071000179701002328F7986FF01FF8BB
:107C2000979701009387479883A70700179701004C
:107C3000232E0796E39C07F29797010093874798B6
:107C400083A707009387170017970100232AF79649
:107C50006FF0DFF1179701001307079783280700DC
:107C600097970100938707968325070017960100D1
:107C70001306069383A60700032606001798010043
:107C8000130848920327080017950100232CB5908C
:107C9000130500006306D600330717413335E000B3
:107CA00003A6070017970100130787919797010014
:107CB0009387C78E8326070083A707000327070043
:107CC0009795010023AEC58CB387D740B337F0003A
:107CD000B307F0409796010023A2E68C3375F500B8
:107CE00067800000B305B500930705006386B70001
:107CF00003C70700631607003385A74067800000AD
:107D0000938717006FF09FFE130101FB232291045C
:107D1000232C4103232291032326110423248104CD
:107D200023202105232E3103232A51032328610315
:107D300023267103232481032320A103232EB101D1
:107D4000930C0500138A05009304000063DE050010
:107D50003305A0403337A000B305B040930C0500B5
:107D6000338AE5409304F0FF63DA06003306C0402F
:107D7000B337C000B306D040B386F640930A06007E
:107D80009389060013840C0013090A0063960628E1
:107D9000178B0100130B0B526370CA16B707010053
:107DA0006372F6149307F00F63F4C7009309800021
:107DB000B3573601330BFB0083470B00130500025A
:107DC000B3873701B309F540638C0900B3153A0155
:107DD000B3D7FC00B31A360133E9B70033943C0142
:107DE00013DB0A0193050B0013050900EF00507C1B
:107DF000130A050093050B00939B0A011305090064
:107E0000EF00907693DB0B019305050013850B00C3
:107E1000EF00D072131A0A0193570401B367FA00F6
:107E200063FAA700B387570163E6570163F4A7001D
:107E3000B38757013389A74093050B001305090049
:107E4000EF001077130A050093050B0013050900D6
:107E5000EF0090711314040193050500131A0A0131
:107E600013850B0013540401EF00506D33648A0036
:107E7000637AA40033045401636654016374A4005C
:107E8000330454013304A4403354340193050000F7
:107E9000638A040033048040B3378000B305B040E8
:107EA000B385F540130504008320C1040324810435
:107EB00083244104032901048329C103032A810384
:107EC000832A4103032B0103832BC102032C81026C
:107ED000832C4102032D0102832DC10113010105F1
:107EE00067800000B707000193090001E362F6EC28
:107EF000930980016FF0DFEB631A06009305000021
:107F000013051000EF005066930A0500B707010043
:107F100063FAFA0E9307F00F63F457019309800098
:107F2000B3D73A01330BFB0083470B001305000264
:107F300033095A41B3873701B309F540E38209EAAF
:107F4000B39A3A01335BFA00B3153A01B3D7FC0098
:107F500093DB0A0133E9B70013050B0093850B008F
:107F6000EF001065130A050093850B00139C0A01AE
:107F700013050B00EF00505F135C0C019305050027
:107F800013050C00EF00905B131A0A0193570901C7
:107F9000B367FA0033943C0163FAA700B387570133
:107FA00063E6570163F4A700B3875701338BA740FB
:107FB00093850B0013050B00EF00905F130A05007B
:107FC00093850B0013050B00EF00105A9305050075
:107FD00013050C00EF00905693160901131A0A01BD
:107FE00093D60601B366DA0063FAA600B38656019B
:107FF00063E6560163F4A600B38656013389A640B2
:108000006FF01FDEB707000193090001E3EAFAF001
:10801000930980016FF0DFF06376DA0093050A00C0
:108020006FF01FE7B707010063FAF604930BF00F38
:1080300033B5DB001315350033D7A6009787010051
:1080400093874727B387E70083CB07009305000298
:10805000B38BAB00338B7541631C0B0263E44601A9
:1080600063EACC003384CC40B306DA4033B98C00E9
:1080700033892641930509006FF09FE1B70700019E
:1080800013050001E3EAF6FA130580016FF0DFFA49
:10809000B3966601335D7601336DDD00B35D7A0121
:1080A000B3156A0133DC7C0113540D01336CBC0041
:1080B00013850D0093050400B3196601EF00504FBE
:1080C000930A05009305040013850D0033996C0194
:1080D000931C0D01EF00504993DC0C01130A0500BD
:1080E0009305050013850C00EF005045939A0A0193
:1080F00013570C0133E7EA00930D0A00637EA700D3
:108100003307A701930DFAFF6368A7016376A70001
:10811000930DEAFF3307A701330AA7409305040034
:1081200013050A00EF00D04893050400930A0500E8
:1081300013050A00EF0050439305050013040500E2
:1081400013850C00EF00903F93150C01939A0A01E0
:1081500093D50501B3E5BA001307040063FEA5003B
:10816000B385A5011307F4FF63E8A50163F6A50035
:108170001307E4FFB385A501939D0D01B70C010022
:10818000B3EDED001384FCFFB3F78D0033F48900E9
:10819000338AA54013850700930504002326F100C8
:1081A00093DD0D01EF00903993050400930A05005B
:1081B00013850D00EF00903813DC090193050C00C6
:1081C0002324A10013850D00EF0050378327C10041
:1081D00013040C0093050400130C0500138507001D
:1081E000EF00D0358326810013D70A013305D5006F
:1081F0003307A7006374D700330C9C01B707010055
:108200009387F7FF935507013377F700131707019B
:10821000B3F7FA00B3858501B307F7006366BA00C8
:10822000631EBA00637CF90033863741B3B7C700D9
:10823000B385A541B385F54093070600B307F94020
:108240003339F900B305BA40B3852541339475013C
:10825000B3D767013364F400B3D565016FF05FC332
:10826000130101FD23229102232A51012326110229
:108270002324810223202103232E3101232C4101B9
:1082800023286101232671012324810123229101E6
:108290002320A101930A050093840500639E0638FC
:1082A00013040600930905001789010013098900CA
:1082B00063F8C512B7070100138B05006378F61049
:1082C0001307F00F3337C70013173700B357E60013
:1082D0003309F900834609003387E600930600025C
:1082E000B386E640638C0600B394D40033D7EA002B
:1082F0003314D600336B9700B399DA00935A040114
:1083000093850A0013050B00EF00902A130905005E
:1083100093850A00931B040113050B00EF00D02482
:1083200093DB0B01930405009305050013850B00F7
:10833000EF00D0201319090193D70901B367F900A1
:10834000138A040063FEA700B3878700138AF4FF33
:1083500063E8870063F6A700138AE4FFB38787000A
:10836000B384A74093850A0013850400EF005024CE
:108370001309050093850A0013850400EF00D01E41
:108380009399090193040500930505001319090148
:1083900013850B0093D90901EF00501AB369390115
:1083A0001386040063FCA900B30934011386F4FFAB
:1083B00063E6890063F4A9001386E4FF13140A013D
:1083C0003364C400130A00006F000013B7070001F4
:1083D00013070001E36CF6EE130780016FF01FEF47
:1083E000138A0600631A06009305000013051000A7
:1083F000EF00901713040500B7070100637EF41225
:108400009307F00F63F48700130A8000B357440109
:108410003309F900034709009306000233074701B7
:10842000B386E64063940612B3848440130A1000B6
:10843000135B040193050B0013850400EF00501734
:108440001309050093050B0013850400931B040119
:10845000EF00901193DB0B019304050093050500D9
:1084600013850B00EF00900D1319090193D7090133
:10847000B367F900938A040063FEA700B3878700FF
:10848000938AF4FF63E8870063F6A700938AE4FF0A
:10849000B3878700B384A74093050B0013850400BE
:1084A000EF0010111309050093050B00138504005C
:1084B000EF00900B939909019304050093050500C3
:1084C0001319090113850B0093D90901EF00100757
:1084D000B36939011386040063FCA900B3093401B0
:1084E0001386F4FF63E6890063F4A9001386E4FFB2
:1084F00013940A013364C4001305040093050A00B1
:108500008320C10203248102832441020329010242
:108510008329C101032A8101832A4101032B01011F
:10852000832BC100032C8100832C4100032D01000B
:108530001301010367800000B7070001130A00015F
:10854000E366F4EC130A80016FF05FEC3314D4009F
:1085500033DAE400B399DA0033D7EA00935A04011E
:10856000B394D40093850A0013050A00336B970077
:10857000EF0010041309050093850A0013050A0093
:10858000931B0401EF00407E93DB0B019304050075
:108590009305050013850B00EF00407A13190901BC
:1085A00013570B013367E900138A0400637EA700A9
:1085B00033078700138AF4FF636887006376A70098
:1085C000138AE4FF33078700B304A74093850A00AA
:1085D00013850400EF00C07D1309050093850A0090
:1085E00013850400EF00407893040500930505000F
:1085F00013850B00EF00807413170B01135707014D
:1086000013190901B367E9001387040063FEA7008B
:10861000B38787001387F4FF63E8870063F6A7003A
:108620001387E4FFB3878700131A0A01B384A740B6
:10863000336AEA006FF0DFDF63ECD51EB707010095
:1086400063F4F6041307F00FB335D70093953500A4
:1086500033D7B600978701009387C7C5B387E70074
:1086600003C70700130A00023307B700330AEA40C2
:1086700063160A0213041000E3E096E833B6CA005A
:10868000134416006FF05FE7B70700019305000180
:10869000E3E0F6FC930580016FF09FFBB35CE6001E
:1086A000B3964601B3ECDC0033D4E40093DB0C0159
:1086B000B397440133D7EA0093850B0013050400F8
:1086C000336BF700B3194601EF00806E1309050004
:1086D00093850B0013050400139C0C01EF00C06888
:1086E000135C0C01930405009305050013050C00B1
:1086F000EF00C0641319090113570B013367E90038
:1087000013840400637EA700330797011384F4FFEA
:10871000636897016376A7001384E4FF330797012A
:10872000B304A74093850B0013850400EF00406855
:108730001309050093850B0013850400EF00C06248
:10874000930405009305050013050C00EF00005F7E
:1087500093170B011319090193D70701B367F900A8
:108760001386040063FEA700B38797011386F4FF06
:1087700063E8970163F6A7001386E4FFB3879701C8
:1087800013140401B70B01003364C4001389FBFF09
:10879000337D240133F92901B384A74093050900EF
:1087A00013050D00EF008059935C04019305090047
:1087B000130B050013850C00EF00405893D90901F5
:1087C000130C05009385090013850C00EF0000577A
:1087D000130905009385090013050D00EF000056ED
:1087E0003305850193570B013385A7006374850119
:1087F0003309790193570501B387270163E6F40232
:10880000E392F4BCB70701009387F7FF3375F500D7
:1088100013150501337BFB0033964A0133056501CF
:10882000130A0000E37AA6CC1304F4FF6FF09FB99B
:10883000130A0000130400006FF01FCC130101FBAA
:108840002324810423229104232E31032322910324
:108850002326110423202105232C4103232A51031D
:108860002328610323267103232481032320A103EA
:10887000232EB101930C0500938905001304050014
:1088800093840500639E062613090600138A0600DA
:10889000978A0100938A0AA263F4C514B7070100FE
:1088A0006376F6129307F00F63F4C700130A800093
:1088B000B3574601B38AFA0003C70A001305000242
:1088C00033074701330AE540630C0A00B3954901B9
:1088D00033D7EC0033194601B364B70033944C012D
:1088E000935A090193850A0013850400EF00404C58
:1088F0009309050093850A00131B090113850400E1
:10890000EF008046135B0B019305050013050B0078
:10891000EF00C0429399090193570401B3E7F900AE
:1089200063FAA700B387270163E6270163F4A70072
:10893000B3872701B384A74093850A0013850400F9
:10894000EF0000479309050093850A001385040092
:10895000EF00804113140401930505009399090168
:1089600013050B0013540401EF00403D33E489006C
:10897000637AA40033042401636624016374A400B1
:10898000330424013304A44033554401930500000B
:108990008320C104032481048324410403290104A6
:1089A0008329C103032A8103832A4103032B010383
:1089B000832BC102032C8102832C4102032D01026F
:1089C000832DC1011301010567800000B707000175
:1089D000130A0001E36EF6EC130A80016FF05FEDFD
:1089E000631A06009305000013051000EF00C0375E
:1089F00013090500B7070100637AF90E9307F00F1A
:108A000063F42701130A8000B3574901B38AFA00BF
:108A100003C70A0013050002B38429413307470145
:108A2000330AE540E30E0AEA33194901B3DAE900F3
:108A3000B395490133D7EC0093540901336BB70068
:108A400013850A0093850400EF0080369309050022
:108A500093850400931B090113850A00EF00C030C1
:108A600093DB0B019305050013850B00EF00002D30
:108A70009399090193570B01B3E7F90033944C0123
:108A800063FAA700B387270163E6270163F4A70011
:108A9000B3872701B38AA7409385040013850A0092
:108AA000EF000031930905009385040013850A0047
:108AB000EF00802B9305050013850B00EF000028C5
:108AC00093150B019399090193D50501B3E5B900FD
:108AD00063FAA500B385250163E6250163F4A500CB
:108AE000B3852501B384A5406FF09FDFB707000170
:108AF000130A0001E36AF9F0130A80016FF0DFF056
:108B0000E3E8D5E8B707010063FCF604930BF00F28
:108B100033B5DB001315350033D7A6009777010076
:108B200093874779B387E70083CB0700930500025B
:108B3000B38BAB00338B7541631E0B0263E43601CC
:108B400063EACC003384CC40B386D94033B58C0083
:108B5000B384A64013050400938504006FF05FE31F
:108B6000B707000113050001E3E8F6FA13058001D9
:108B70006FF09FFAB3966601335D7601336DDD00C9
:108B800033D47901B395690133DC7C0193540D0131
:108B9000336CBC001305040093850400B31A66010E
:108BA000EF000021130A050093850400130504005B
:108BB00033996C01931C0D01EF00001B93DC0C0139
:108BC000130405009305050013850C00EF00001742
:108BD000131A0A0113570C013367EA00130A040041
:108BE000637EA7003307A701130AF4FF6368A70198
:108BF0006376A700130AE4FF3307A701B309A74070
:108C00009385040013850900EF00801A9385040002
:108C10001304050013850900EF00001593050500F6
:108C20009304050013850C00EF00401193150C010F
:108C30001314040193D50501B365B4001387040030
:108C400063FEA500B385A5011387F4FF63E8A501C2
:108C500063F6A5001387E4FFB385A501131A0A0183
:108C6000B70C0100336AEA001384FCFFB3778A0073
:108C700033F48A00B384A5401385070093050400EC
:108C80002326F100135A0A01EF00400B9309050057
:108C90009305040013050A00EF00400A13DC0A01E3
:108CA000930D050093050C0013050A00EF00000961
:108CB0008327C100130A050093050C0013850700E4
:108CC000EF00C0073305B50113D709013307A7002B
:108CD0006374B701330A9A01B70701009387F7FF5E
:108CE000935507013377F70013170701B3F7F9001E
:108CF000B3854501B307F70063E6B400639EB40093
:108D0000637CF90033865741B3B7C700B385A541EB
:108D1000B385F54093070600B307F9403339F900EE
:108D2000B385B440B385254133947501B3D767014A
:108D30003365F400B3D565016FF09FC513060500D8
:108D40001305000093F61500638406003305C50083
:108D500093D5150013161600E39605FE67800000F4
:108D60006340050663C605061386050093050500E6
:108D70001305F0FF630C060293061000637AB60039
:108D80006358C0001316160093961600E36AB6FEE9
:108D90001305000063E6C500B385C5403365D50003
:108DA00093D6160013561600E39606FE6780000061
:108DB00093820000EFF05FFB1385050067800200DF
:108DC0003305A04063D80500B305B0406FF0DFF96C
:108DD000B305B04093820000EFF01FF93305A040C7
:108DE000678002009382000063CA0500634C05009F
:108DF000EFF09FF71385050067800200B305B040D0
:108E0000E35805FE3305A040EFF01FF63305B040F0
:108E100067800200977701009387077583A6070094
:108E200017770100130707730327070023A2A60083
:108E3000637EE5001777010013078772032507009B
:108E400083A50700938545006F70DF93130101FF31
:108E50002324810023261100177701001307877050
:108E6000130405000325070083A50700938545002B
:108E7000EF705F91977701009387076C83A70700D6
:108E80006376F4009777010023A8876A8320C100E6
:108E9000032481001301010167800000977701001E
:108EA0009387876C03A7070083A6070083274704DF
:108EB0009387F7FF2322F70483A7460463940700F0
:108EC0007360043067800000130101FE232C8100D1
:108ED000232A91001304050093840500232821010F
:108EE000232631012324410123225101232E110085
:108EF000EF909FC58327040003290401B7090001EF
:108F0000B3E59700930AC4002320B4009304000043
:108F10009389F9FF370A00020327040063822A05B8
:108F20000326090013050900B3654701B37636012E
:108F30009317560033F7E6000329490063C607007C
:108F4000631607006FF05FFDE398E6FC9317760069
:108F500063D40700B3E4D400EFB04F876FF0DFFBBA
:108F600093C4F4FFB3F4E40023209400EF905FF186
:108F7000032504008320C1010324810183244101CE
:108F8000032901018329C100032A8100832A4100AA
:108F90001301010267800000130101FF2326110065
:108FA00023248100EFE08F9B17E7FFFF1307C70A19
:108FB0009306000013061000930540061775010084
:108FC00013054544EFC08FB8630205021304050082
:108FD000EF901FB913060500130700009306000069
:108FE0009305100013050400EFC04FC8EF901F83D6
:108FF0008320C10003248100130500001301010137
:049000006780000085
:02000004800278
:100000004064FEFFB065FEFF4C64FEFFB065FEFF7E
:10001000B065FEFFB065FEFFB065FEFF7464FEFFD5
:10002000B065FEFFB065FEFF9C64FEFFAC64FEFFA2
:10003000B065FEFFC464FEFFD464FEFFD464FEFF1F
:10004000D464FEFFD464FEFFD464FEFFD464FEFFDC
:10005000D464FEFFD464FEFFD464FEFFB065FEFFEF
:10006000B065FEFFB065FEFFB065FEFFB065FEFF48
:10007000B065FEFFB065FEFFB065FEFFB065FEFF38
:10008000B065FEFFB065FEFFB065FEFFB065FEFF28
:10009000B065FEFFB065FEFFB065FEFFB065FEFF18
:1000A000B065FEFFB065FEFFB065FEFFB065FEFF08
:1000B000B065FEFFB065FEFFB065FEFFB065FEFFF8
:1000C000B065FEFFB065FEFFB065FEFFB065FEFFE8
:1000D000B065FEFFB065FEFFB065FEFFB065FEFFD8
:1000E000B065FEFFB065FEFFB065FEFFB065FEFFC8
:1000F000B065FEFFB065FEFFB065FEFFB065FEFFB8
:100100001865FEFF4065FEFFB065FEFFB065FEFFAF
:10011000B065FEFFB065FEFFB065FEFFB065FEFF97
:10012000B065FEFFA065FEFFB065FEFFB065FEFF97
:100130005062FEFF5863FEFFB065FEFFB065FEFF34
:10014000A863FEFFB065FEFF2064FEFFB065FEFF02
:10015000B065FEFF6864FEFF0C6AFEFF786AFEFF72
:10016000186AFEFF786AFEFF786AFEFF786AFEFF73
:10017000786AFEFFB068FEFF786AFEFF786AFEFFCD
:10018000D868FEFFE868FEFF786AFEFF0069FEFFA0
:100190001069FEFF1069FEFF1069FEFF1069FEFF87
:1001A0001069FEFF1069FEFF1069FEFF1069FEFF77
:1001B0001069FEFF786AFEFF786AFEFF786AFEFF2C
:1001C000786AFEFF786AFEFF786AFEFF786AFEFFB3
:1001D000786AFEFF786AFEFF786AFEFF786AFEFFA3
:1001E000786AFEFF786AFEFF786AFEFF786AFEFF93
:1001F000786AFEFF786AFEFF786AFEFF786AFEFF83
:10020000786AFEFF786AFEFF786AFEFF786AFEFF72
:10021000786AFEFF786AFEFF786AFEFF786AFEFF62
:10022000786AFEFF786AFEFF786AFEFF786AFEFF52
:10023000786AFEFF786AFEFF786AFEFF786AFEFF42
:10024000786AFEFF786AFEFF786AFEFF786AFEFF32
:10025000786AFEFF786AFEFF5469FEFF9069FEFF30
:10026000786AFEFF786AFEFF786AFEFF786AFEFF12
:10027000786AFEFF786AFEFF786AFEFFFC69FEFF7F
:10028000786AFEFF786AFEFF8466FEFFD867FEFF8D
:10029000786AFEFF786AFEFF6868FEFF786AFEFFF4
:1002A0009468FEFF786AFEFF786AFEFF6C6AFEFFC4
:1002B000000102020303030304040404040404040D
:1002C00005050505050505050505050505050505DE
:1002D00006060606060606060606060606060606BE
:1002E00006060606060606060606060606060606AE
:1002F000070707070707070707070707070707078E
:10030000070707070707070707070707070707077D
:10031000070707070707070707070707070707076D
:10032000070707070707070707070707070707075D
:10033000080808080808080808080808080808083D
:10034000080808080808080808080808080808082D
:10035000080808080808080808080808080808081D
:10036000080808080808080808080808080808080D
:1003700008080808080808080808080808080808FD
:1003800008080808080808080808080808080808ED
:1003900008080808080808080808080808080808DD
:1003A00008080808080808080808080808080808CD
:1003B000546D725100000000546D7220537663003A
:1003C000286E756C6C2900004572726F7220696E20
:1003D00020787878207461736B73200D0A00000018
:1003E0006D69616F750A00006D69616F75320A0091
:1003F00068756E6772790A0054696D657232000023
:10040000436865636B54696D657200005761697478
:100410004F0000005365744200000000526E647685
:0404200000000000D8
:100424001000000000000000017A5200017C01016C
:100434001B0D02005000000018000000C878FEFFE9
:100444005805000000440E507489039406990B81EA
:1004540001880292049305950796089709980A9AC9
:100464000C9B0D036C010AC144C844C944D244D353
:1004740044D444D544D644D744D844D944DA44DB9C
:10048400440E00440B0000004C0000006C0000000F
:10049400CC7DFEFFDC05000000440E30708903951E
:1004A4000781018802920493059406960897099897
:1004B4000A990B9A0C0370020AC144C844C944D275
:1004C40044D344D444D544D644D744D844D944DA54
:1004D400440E00440B00000050000000BC0000006B
:1004E4005883FEFF0005000000440E507488028902
:1004F400039305990B810192049406950796089736
:1005040009980A9A0C9B0D0320010AC144C844C9E6
:1005140044D244D344D444D544D644D744D844D90B
:0C05240044DA44DB440E00440B000000ED
:0805C800FC8F01000900000096
:040000058000004037
:00000001FF
